:10000000F01F00108D4900008B4900008B49000053
:100010008B4900008B4900008B4900000000000064
:100020000000000000000000000000008B490000FC
:100030008B490000000000008B490000C51E000035
:10004000DD1C0000DD1C0000DD1C0000DD1C0000CC
:10005000DD1C0000DD1C0000DD1C0000DD1C0000BC
:10006000DD1C0000DD1C0000DD1C0000DD1C0000AC
:10007000DD1C00008949000089490000C100000022
:100080008D1F0000A51F0000B9210000D121000034
:1000900089490000152300008949000089490000B2
:1000A0008949000089490000894900008949000008
:1000B00089490000894900008949000089490000F8
:1000C000554B10B51A6801321A60544B1A68544BDC
:1000D000D2B2302A69D01ADC182A44D012DC082A9D
:1000E00032D0102A00D094E04E4A002111604E49CF
:1000F0000A68501C08604D49895C4D4AC9B21160BC
:10010000282287E0202A63D0282A32D081E0482A9A
:100110005ED004DC382A51D0402A53D079E0502AEE
:1001200060D0582A75D13F490A68501C0860404980
:1001300008684049C0B288543F4A0221FF3111602B
:1001400080221021D20563E0374A00211160116836
:10015000481C1060354A515C354AC9B211602822EA
:100160001A6001223CE030490A68501C08602F499F
:1001700009E02D4A314910680968884207D21168A0
:10018000481C1060294A515C294AC9B240E02C4AF7
:1001900011688022D205002901D0202138E02649AB
:1001A0000220FF300860102132E08022D2051021A9
:1001B000116008221A608122520011E08221490058
:1001C0001D4A25E01E4A1168042201291AD11DE0AA
:1001D0008022D2051021116008221A600422FF3209
:1001E000154B17E00F4A1168481C1060104804684E
:1001F0001048E4B244541068114A116804220139CD
:10020000884203D28021C9050A6002E01A6000E03A
:10021000116008221A6010BD8C0300100400004019
:10022000180000408003001088030010A005001093
:10023000080000409005001084030010B005001075
:100240008C0500101B4B02211A6810B50A431A6076
:10025000194B20211A68041C0A431A60174B1849CD
:100260001A680A401A601868012210431860154B7A
:1002700018680140196019680A431A60124B6C2211
:100280001A60124B1249186804F006FC114A1060FB
:10029000114A1060022C02D1104BA0221A60104BA0
:1002A000802212021A6080234022DB0501201A609E
:1002B00010BDC046048004408080044030400440AB
:1002C000F8FCFFFF34400440180000408405001093
:1002D000400D030014000040100000400C000040DE
:1002E00000E100E0034B1B689A06FBD5024B186047
:1002F0007047C0461480004000800040FFFFFFFFB1
:1003000070B5061C00200D1C00F0EEFF002801D087
:1003100002F0CEFB00242C60301C3460291C01F05C
:1003200011F8201C00F0E0FFA04207D002F0C0FB53
:100330002C60301C3460291C01F004F870BD08B535
:1003400001F0F0FD08BD08B500230B60036000F06C
:10035000F9FF08BD10B502F073FB0D4B00201968C2
:1003600001F0A0FF002001F08DFF002001F06AFFE6
:10037000084B01241C60084B201C198801F04EFE1C
:10038000201C01F03BFE201C01F018FE10BDC046F1
:10039000800500107C0300108805001008B50A20B5
:1003A000002101F08BFDFFF7D5FF08BD08B5002047
:1003B00001F058FF012001F011FE02F047FB08BDDB
:1003C00038B5051C0C1CFFF7C5FF054B0122281C86
:1003D000211C5A6203F000FEFFF7E8FF38BDC0465B
:1003E0005C0D001010B5041CFFF7B4FF201C03F0D7
:1003F0007BFD041CFFF7DAFF201C10BD08B50020B0
:10040000FFF7F0FF08BD000008B5021C02490348D1
:1004100002F0A6F908BDC046C84B0000C04B000062
:1004200037B500F0D7FD0322164B1748002100F026
:10043000BFFE00F0D9FDFFF7E1FF1448FFF7E4FF2E
:10044000134B144A00241A601D1C2B689C4211DABD
:1004500002F042F8002803D001F01CFB00240FE05A
:100460000A2001F05FFD684601A9FFF749FF009BE4
:10047000002B05D0FFF7C2FF074802F071F937BD26
:100480000134E2E708000010CD4B0000DC4B000017
:100490007004001070170000E24B0000704700006D
:1004A0001B4B73B5041C1B49186804F0F5FA1A4974
:1004B00000901A4A1A4B201C02F05EF901F01EF857
:1004C000002812D001F036F8FA218900061C04F049
:1004D000E3FA051C201C02F0A0F9124B20186B4314
:1004E0001149F3182A1C02F047F9201C02F095F973
:1004F0000E4B20181B68002B02D003DA0C4A02E0D6
:100500000C4A00E00C4A0D4902F036F973BDC046B2
:100510008405001040420F00F34B0000C84B000060
:10052000004C000018FCFFFF044C000050020010BB
:10053000F04B0000ED4B0000849300000F4C0000D6
:1005400070B5051C0E1C141C00F044FD301C291C49
:100550000022064B00F02CFE201C01210922044B36
:1005600000F026FE00F040FD70BDC04608000010FF
:100570001400001000B5084B89B01A78074B684684
:100580001B78074902F0F8F801206946054AFFF791
:10059000D7FF09B000BDC046440200101000001093
:1005A000434C0000514C0000F0B52A4C2A4D2378F2
:1005B00085B001932F78FFF7DDFFFFF71FFF0026BF
:1005C00002A803A9FFF79CFE029800282BD0C0B216
:1005D00000F008FE40280CD004D830280ED039286E
:1005E00017D01BE0462830D049280DD0412815D11E
:1005F00026E02B783E2B11D8013303E02B78002B1B
:100600000CD0013B2B7009E02378062B06D8013370
:1006100003E02378002B01D0013B237000F0C6FCDF
:10062000FFF7A8FF0026029B002B02D0C82001F094
:1006300079FC04200321013601F040FC1D2EBFDDB2
:10064000019B2F70237000F0B1FCFFF7D7FE05B0BF
:10065000F0BDC046100000104402001010B590B06C
:10066000041C6846FFF71CFF201C69466A46FFF71A
:1006700067FF10B010BD000000B52D228DB000281E
:1006800000D02B2268460D4902F076F804A802F04B
:10069000A1FA0120694604AAFFF752FF03200021B6
:1006A00001F00CFC0220FFF79DFE0028EED00A208E
:1006B000002101F003FC0DB000BDC046654C0000F8
:1006C00070B58CB0FFF79AFE02A8144902F0AEF89C
:1006D0002E25FF3504AE301C02F07CFA684600245B
:1006E00009A90930F47402F0A1F802AA0420311C0F
:1006F000FFF726FF201C032101F0E0FB684601A95B
:1007000001940094FFF7FCFD009BA34202D1013D40
:10071000A542DFD1FFF772FE0CB070BD85930000DB
:10072000F7B502F0EDF918200021FFF749FE00248B
:10073000664EFFF73BFE664D00236B62201C02F005
:1007400000FA002C02D00020012101E00620032144
:1007500001F0B4FB201C02F0EFF901A9071C684668
:10076000002F03D0FFF7EFFD012728E0FFF7EBFD97
:10077000009A002A23D1002CE0D1564F3B1C98331D
:100780001B68002B0DD1544BF618D7D5182000212B
:100790009437FFF715FE3C6863425C4100F0CEFBE6
:1007A000CCE74E4B00941A6811321A60009A102A56
:1007B000E9DC03F049FB009B01330093F6E7002CD2
:1007C0000CD0009B182B01D0002FB2D000F014FCED
:1007D0004348FFF719FE3F4B0122DA6600F0BCFEEA
:1007E00002F0F8F8009A182A59D1019F0024F8B2B3
:1007F00000F0F8FC012601946E6217283DD00CD859
:10080000132827D002D811281CD045E0152824D061
:10081000162841D1FFF7C8FE41E0262825D007D889
:10082000192839D12F4B1868301A00F0A9FF14E0AD
:1008300044282AD045282FD1E120000102F052FAA5
:10084000301C26E0284B1B68002B28D0FFF738FF10
:10085000009424E0FFF7E4FD21E00120FFF7FEFE15
:10086000FFF7CCFDFFF79AFD19E0204B05221C7025
:100870001F4B1A7000F09AFB11E01E4B1A680132F0
:100880001A60032A0BD11C6009E01B4802F02AFA07
:10089000201CFFF7F1FE02E0002301976B62FFF7D7
:1008A00059FD0098019903F097FB6B6A002B01D06A
:1008B000FFF7A4FD074B94331B68002B03D100F016
:1008C0003DFB012434E703F0FFFF30E720BF0200C7
:1008D0005C0D0010C00500100CFEFFFF900300101F
:1008E0006E4C000020000010500200104402001066
:1008F000100000101C020010F0F1FFFF73B501F0B2
:10090000D3FF3A4C00F0B2FC3948002101F05AF90B
:100910000021384801F056F900F080FD00F00EFF8C
:1009200023680726B3432360236801252B43002057
:100930002360021C0B2101F0CFF8201C2E4C10214B
:1009400001F040F923680022B34323602368281C88
:100950002360042101F0C0F8201C002101F032F9CD
:1009600001F0A4F89620000201F012FD234D0123AE
:100970005B4200202B60FFF771FE00232B605024A8
:100980000120FFF75FFC00F0D9FE02F083F82B682E
:10099000002B05D16420043C01F0C4FA142CEFD1E3
:1009A0000020FFF75BFE164801F0DAFE192001F087
:1009B000B9FA01F091FD002802D0FFF731FD02E005
:1009C000013C002CF2DC02F0A1FA03F05DF91E23D9
:1009D00000930F2301930B480B4900220B4B03F0AC
:1009E00065F90B4803F094F9FFF79AFE7440044050
:1009F000984004409C400440944004405002001041
:100A0000784C0000454900000103000090030010ED
:100A10007C030010F7B500283BD00378303B5A42E6
:100A20005341C0180378782B03D1013010260125DB
:100A300001E00A2600250378002201922D2B02D125
:100A400001230130019300230278002A1BD0171CD8
:100A5000303FFCB2092C02D87343DB1911E0202788
:100A60003A43002D08D0171C613FFFB2052F03D871
:100A70001B01573A134304E0064801F071FE0020C1
:100A800007E00130E0E7019A002A00D05B420B60EA
:100A90000120FEBD824C00000378202B01D10130E3
:100AA000FAE77047031C303BDAB2092A01D8181C58
:100AB0000AE020231843031C613BDBB2052B01D85D
:100AC000573801E001204042704770B50E1CFFF717
:100AD000E3FF0025041C2078002807D0FFF7E2FF81
:100AE000002803DB2D0105430134F4E73560201CA9
:100AF00070BD000008B500F01DFD011C014801F0AB
:100B00002FFE08BD904C000000B589B0684602F089
:100B100061F86946024801F023FE09B000BDC046F5
:100B2000CC4C0000F7B50F1C01A9161CFFF772FF93
:100B3000002814D0019C0B49201C04F003F80D1C64
:100B4000081C642103F0FEFF281C3970642103F0A7
:100B5000A3FF04493070201C03F09EFF01E0012038
:100B60004042FEBD1027000037B50D1C48686A469C
:100B7000694607310632FFF7D5FF01AC69466A4680
:100B800020800132A8680231FFF7CCFF6B46187055
:100B90002288044B9A4203D9201C694602F088F847
:100BA00037BDC0466B07000007B5486801A9FFF7CD
:100BB00031FF019B3C20584302F094F807BD000030
:100BC00007235843054A10189C30013B04D3C25CEC
:100BD000002AFAD0002000E001207047C005001074
:100BE00030B5194885B001F0BBFD0024651CA30792
:100BF00019D1201CFFF7E4FF002810D0281CFFF7B4
:100C0000DFFF00280BD0A01CFFF7DAFF002806D07A
:100C1000E01CFFF7D5FF002801D004340EE00B489C
:100C2000211C01F09DFD211C684602F083F96846F5
:100C300001F054FE064801F093FD2C1CFF2CD5DD7D
:100C400001F05AFE05B030BDC84B00009C4C0000BE
:100C50008493000070B50E1CFFF71EFF0D25041CC9
:100C60000134631E1878FFF71DFF002806DB70555E
:100C7000013DF5D2201CFFF70FFF00E0002070BD02
:100C800070B5424C86B023680868251C002B06D13D
:100C90003F4801F065FD02F0F7FF012351E0012B11
:100CA0000CD13C49042201F0CAFD002802D123687E
:100CB000013346E0384801F053FD5CE00378412BF6
:100CC0001BD1364C0230211CFFF7C4FF002852D044
:100CD0000378422B4FD1211C02300E31FFF7BAFFAF
:100CE000002848D00378432B45D1211C02301C3109
:100CF000FFF7B0FF002846D13DE04D2B23D1284E11
:100D00000230311CFFF7A6FF002834D003784E2BA9
:100D100031D1311C02300E31FFF79CFF00282AD060
:100D20000378472B27D1023001A9FFF7CEFE019BA4
:100D3000002B20DB2A3E1B481B49736501F010FD88
:100D4000002323601FE001A9FFF7BFFE04782023E2
:100D5000061C9C430FD1301C02A9FFF77BFF019BAF
:100D6000061CE11802A802F0FBF8002E03D00134A3
:100D7000042CF0D107E002F087FF0A480B4901F08C
:100D8000EFFC00232B6006B070BDC046540300107A
:100D9000A54C0000C84B0000BB4C0000C005001073
:100DA000EA050010C74C0000214C0000D14C0000A7
:100DB00037B54C682378002B25D0201CFFF76CFE3C
:100DC00001A9FFF782FE019B041C002B1BD0D8B2A7
:100DD000FF2B09DD00F022FA019B051C1812C0B29E
:100DE00000F01CFA019003E000F018FA00250190D1
:100DF0000198002802D0291CFFF7E2FA23785A1E36
:100E00009341E418D6E737BD064A08B513780121A7
:100E10004B40137001D0044900E00449044801F03C
:100E20009FFC08BD74040010754C0000D84C0000F5
:100E3000DC4C000007B5486801A9FFF7EBFD019BFA
:100E4000002B01DC01230193019B1E2B01DD1E23DE
:100E500001930199034A044B4A4304481A6001F084
:100E60007FFC07BD7017000070040010EB4C000001
:100E700038B5051C002D09D0642402200021013C56
:100E800000F050FE002CF8D1013DF3E738BD70B5FD
:100E9000061C01200821021C00F06EFE0724012020
:100EA0000821002200F068FE321C012522412A4060
:100EB0000020022100F060FE281C08212A1C00F0FE
:100EC0005BFE013CEBD270BD10B50021041C0A1C76
:100ED000022000F051FE201CFFF7D9FF10BDF0B535
:100EE000012385B002930023061C039372B60024ED
:100EF00002AB1B59502040421843C0B2FFF7E4FF39
:100F00000020FFF7E1FF1020FFF7DEFFE020FFF7F2
:100F1000DBFF212767430025F7190220002101226A
:100F200000F02AFE785D0135FFF7B1FF842DF4D182
:100F30000434082CDCD162B605B0F0BD08B5AC2095
:100F4000FFF7C2FFAE20FFF7BFFFA520FFF7BCFFF2
:100F500008BD38B50122051C0C1C00F0BDFD281C85
:100F6000211C012200F008FE38BD08B5AF20FFF7B4
:100F7000ABFFA420FFF7A8FF08BD08B5AE20FFF720
:100F8000A3FF08BD10B5041CF820FFF79DFF201C2F
:100F9000FFF79AFF10BD10B5041C8120FFF794FFE6
:100FA0003F202040FFF790FF10BD000008B5074B21
:100FB00020201B781843FFF787FF0A20FFF758FF10
:100FC000034B1878FFF7E7FF08BDC046100000107C
:100FD0004402001008B5842202480021520001F0AA
:100FE000F9FB08BD7504001008B50248FFF777FF4C
:100FF00008BDC0467504001008B501200821FFF7A0
:10100000A8FF00200221FFF7A4FF02200021FFF724
:10101000A0FF02200621FFF79CFF0320011CFFF721
:1010200098FF0320011C002200F0A6FD02200621EB
:10103000002200F0A1FD06210122022000F09CFD0B
:10104000FFF7C8FFFFF7D0FFA220FFF73DFFA0206A
:10105000FFF73AFFC020FFF737FF0020FFF792FFAE
:101060000A20FFF705FF4020FFF72EFF2C20FFF797
:101070002BFF3220FFF7FCFE2E20FFF725FF32204A
:10108000FFF7F6FE2F20FFF71FFF0A20FFF7F0FE05
:10109000FFF78CFFFFF769FF08BD000083280ED81B
:1010A0000F290CD8CB08842253430722C0181140C3
:1010B000034B80220A41111C1A5C114319547047DA
:1010C00075040010F7B55B18DBB20193019B9942E0
:1010D00015D28425CC086C4307270F4080250419BE
:1010E0003D41EFB2A618B44206DA054D65192B78DA
:1010F00001343B432B70F6E70131C9B2E6E7F7BD97
:1011000075040010F0B51E1C87B00592F2780491AA
:101110005B68824201D2307845E0244AB478934239
:1011200005D10322041B54430192E4180CE0001B78
:101130000022824204DA1978013202315B18F8E7A2
:101140001A789C1C5B780193A218002503922F1C2F
:10115000019B9F4226DA08220023029200937378B3
:10116000009A9A421CDA029A082A06D1039B9C42F2
:1011700018D00022257802920134EB0708D5049A92
:10118000009BB818059AC0B29918C9B2FFF786FF3C
:10119000009B029A013301326D1000930292DEE748
:1011A0000137D5E7019807B0F0BDC0460F4D0000EC
:1011B000F7B5041C0D1C161C1F1C01F02EFB20187B
:1011C0000190019B9C420BD0832D09D82078291CCB
:1011D000321C3B1CFFF796FF01302D180134F0E75D
:1011E000F7BD000010B50021012204230A4C0C5D5C
:1011F000844203D118010243D0B20BE0013B002B23
:1012000004D10132092A00DD1A1C042301312829E6
:10121000ECD1002010BDC046BC5400000F230209D1
:1012200018408000031F00D52833511E00200329D9
:1012300006D8242B04DC04218A1A0249CB18985CB6
:101240007047C046BC54000038B5051C0024054B4F
:10125000291CE05C044B0134C01800F0B3FC0A2CDC
:10126000F5D138BDF854000000400440F8B50D4FEA
:101270003C68002C15D11020FFF7E6FF0A4B002236
:10128000E65C1B195D78301C291C00F025FC02343B
:10129000301C291C012200F06FFC142CEED101231C
:1012A0003B60F8BD48020010E454000070B5002413
:1012B0000B4B0122E65C1B195D78301C291C00F0E9
:1012C0000BFC0234301C291C002200F055FC142CAD
:1012D000EED10020FFF7B8FF024B00221A6070BD6C
:1012E000E45400004802001038B5051CFFF7BEFFAB
:1012F000002D09D007210122022000F0EDFB104B48
:1013000080211A688A431A6000200B2100F00AFC31
:101310000124002805D000200B2100F003FC4442EA
:101320004441002D09D007210022022000F0D4FB07
:10133000034B80211A680A431A60201C38BDC0463E
:10134000FC3F0250F0B587B00026029001200391C7
:1013500004960596FFF7C8FFB04202D01823049305
:1013600001260021284C009120786178012200F0AC
:10137000B3FB20786178002200F0FEFB234B9D1D1B
:10138000012E24DC6A782F78111C381C019200F0A1
:10139000C9FB002808D100991D4AB3008A5C1033AC
:1013A00069465A5001360BE02878697800F0BAFB9C
:1013B0000028F0D0381C019900F0B4FB0028EAD0D6
:1013C000009A144B0132023D00929D42D8D12778F9
:1013D0006578381C291C002200F07EFB291C381C73
:1013E000012200F0C9FB0C4902348C42BCD1002020
:1013F000864206D0049A029B05991A60039A01203E
:10140000116007B0F0BDC046E4540000B4540000C1
:10141000BC540000B2540000F854000008B501208C
:10142000021C0B2100F058FB01200B21002200F0D0
:10143000A3FB03200221012200F04EFB0320022126
:10144000002200F099FB08BD234B37B51A68102124
:101450008A431A60214B8022196892010A431A605C
:10146000051C0B210120002200F036FB01200B217E
:10147000002200F081FB1A4B9F211A68194C8A4305
:101480001A601A6818491A60184B186803F004FBB0
:101490008023000218432A1C20600221032000F050
:1014A0006BFB142000F03EFD2368FF229343236072
:1014B00023680F4A134323600E4B1B680193019B63
:1014C000002BF9DA22680C4B13402360FFF7A6FFCC
:1014D00001980004800D3EBD3882044080800440A5
:1014E0009840044000C0014000093D008405001000
:1014F000800000012CC00140FFFFFFF810B50C4C2C
:101500002068002813DA00202060FFF79DFF0A28DA
:101510000ADC0120FFF798FF0138C023FF385B0089
:10152000984201D801232360FFF778FF206810BD9F
:101530001C00001008B5FFF7E1FF002801D10020D2
:1015400007E00120FFF780FF011EF8D0014803F0FB
:10155000A3FA08BD50BB120008B5FFF7CFFF002863
:101560000AD0FFF7E7FFFA22031C0021C00FD200C8
:101570009A424841014B186008BDC0464C02001019
:1015800008B5074B02221A60064BA2221960064BCF
:101590001A70A32258709A7000F0D4FD08BDC0469E
:1015A000B00500108C050010A005001008B5064B12
:1015B00002311960054B00221A60054BA2221A70F5
:1015C000587000F0BFFD08BDB00500108C0500107C
:1015D000A005001070B5051C0E1C0324281C311C2E
:1015E000FFF7CEFF0223FF33984202D0013C002CCC
:1015F000F4D170BD70B5051C0E1C0324281C311CD1
:10160000FFF7D4FF0223FF33984202D0013C002CA5
:10161000F4D170BD0B4B10B51C6800239C420ED05A
:10162000094CA31CA270140A5C70140C120EDA7020
:101630009C70FFF7DFFF831EFF3B5A425341181C8B
:1016400010BDC04650020010A005001070B50E4C31
:1016500025680024A54215D00C4C160AA270E6702D
:10166000160C120E6271A371A21D26711C0A547011
:101670001C0C1B0E9470D370FFF7BCFF841EFF3C44
:1016800063425C41201C70BD50020010A005001098
:1016900008B5064B1A6800239A4205D0FFF79AFF57
:1016A000831EFF3B5A425341181C08BD50020010D4
:1016B00008B5074B00201B68834207D00220072192
:1016C000FFF788FF0238FF384342584108BDC04643
:1016D0005002001008B5074B00201B68834207D05A
:1016E00002200721FFF786FF0238FF3843425841A6
:1016F00008BDC04650020010012010B5011CFFF7C4
:1017000069FF0223FF3398420ED1094B0121196072
:10171000084B1C78230709D0074B032222409A70FC
:10172000081CFFF767FF01E001246442201C10BD84
:101730005002001090050010A005001008B5FFF73A
:10174000DBFF02200121FFF745FF0223FF33984210
:101750000FD1084B1B787F2B06D98422022007214A
:101760005204054BFFF772FF09200421034AFFF7DB
:1017700051FF08BD90050010020114008080808098
:1017800010B500280CD0254B80211A688A431A60B6
:10179000234B1B68D907FBD5224B03221A6001E0BB
:1017A000204B1860204B012200211A6019601A603A
:1017B000196801221142FBD01C4B80211A601C4A7F
:1017C00049021468214311601A1C002804D1134BEC
:1017D0008024196821431960164B196888421CD06F
:1017E0001860002801D0144800E01448116803F084
:1017F00005F9134BFA2118608900041C03F04CF919
:101800001E2358430F4BC82118604901201C03F0C8
:1018100043F90D4B186001F031F810BD38820440D7
:101820000C80044070800440748004407880044040
:101830008080044020000010006CDC02001BB70018
:1018400084050010800500108805001008B500F020
:1018500035F9134B00211A68120B12031A60114B51
:101860001A68120B12031A600F4B1A68120B12033C
:101870001A600E4B1A68120B12031A600C4B0122ED
:1018800019600C4B1A6019601A601A680120024234
:10189000FBD0094B23221A60FFF772FF08BDC04638
:1018A00000800050008001500080025000800350F2
:1018B00040800440448004400880044038B50F490B
:1018C0000F4800F04DFF0F4D0024281C00F048FF8A
:1018D0000D4A0E48A1581219D2682B1C143400F07E
:1018E0003FFFC82CF4D10A4800F03AFF00F03AFB61
:1018F000011C084800F034FF38BDC046C84B00004A
:10190000025500005255000024000010145500003C
:101910001F55000041550000F0B53B4B8BB01E68D1
:10192000041C002E01D1351C08E0384B02901B68C6
:1019300001209B6854E033681E79019D2378002BB9
:1019400031D0082D33D02378202B01D10134FAE790
:10195000002B28D06A1CAD0008356B460192EC5074
:10196000FF2E4CD02278002A07D0631C202A01D0F9
:101970001C1CF7E7002222701C1C019A012ADCD1F2
:10198000224E234B0B253360371C013D002D2ED0FA
:101990003B680298196800F063FF0028CBD03B68D1
:1019A00014333B60F1E7002D1CD0022D02D0B5426C
:1019B00006D911E00398174900F052FF0028F6D12C
:1019C000124C15482368D96800F0CAFE23681348F2
:1019D000196900F0C5FE05E00C4BE8B21B689B6876
:1019E00002A99847084A1368002B0BD103E0281C72
:1019F000291CFFF763FF0A4800F0B2FE02E0019DD8
:101A00000026D2E70BB0F0BD540300105C030010B9
:101A100024000010F14B00004E550000CC4C00009B
:101A20005555000038B5041C164D0A2808D002D8B8
:101A3000082811D01CE00D2802D07F280CD017E018
:101A40002A6800231370104800F08AFE0F4C201CF7
:101A5000FFF762FF2C6013E00C4B2A689A420FD903
:101A60000B48211C00F07CFE2B68013B2B6007E03B
:101A70000748211C00F074FE2B685A1C2A601C7059
:101A800038BDC046580300105255000054020010E3
:101A90006155000008B500F01FFD002804D000F0DB
:101AA000F1FCFFF7BFFFF6E708BD0000014A024B5B
:101AB0001A6070475402001058030010044B402174
:101AC0001A680A431A60034B01221A707047C04615
:101AD00080800440600300100F4B70B51B78061C1B
:101AE0000C1C151C002B01D1FFF7E8FF701E02280B
:101AF00003D80A4B8000C35800E0094B1A68012D37
:101B000004D1A5402C1C14431C6003E00121A1401A
:101B10008A431A6070BDC04660030010485600003A
:101B20000080005038B50F4B051C1B780C1C002B97
:101B300001D1FFF7C3FF0020032D12D8281C01227A
:101B400002F048FF02040608074B04E0074B02E0DE
:101B5000074B00E0074B1B68A2401340181C421EB5
:101B6000904138BD60030010FC3F0050FC3F015025
:101B7000FC3F0250FC3F03500F4B70B51B78061C16
:101B80000C1C151C002B01D1FFF798FF701E0228BA
:101B900003D80A4B8000C35800E0094B1A68012D96
:101BA00004D1A5402C1C14431C6003E00121A1407A
:101BB0008A431A6070BDC04660030010545600008E
:101BC000FC3F005038B5084B041C1B780D1C002B43
:101BD00001D1FFF773FF2368182293432360236822
:101BE0001D43256038BDC04660030010054B3F22F1
:101BF0001A60054B01221A60044B40211A688A437F
:101C00001A60704724800440D88004403882044021
:101C100008B5044B40211A688A431A60FFF7E6FFB3
:101C200008BDC0463882044008B500F051FAFFF7FD
:101C30003DFB0A480021FFF7C5FF09480021FFF7D7
:101C4000C1FF08480021FFF7BDFF07480021FFF74B
:101C5000B9FF06480021FFF7B5FF08BD0840044062
:101C600000400440AC400440144004401C40044088
:101C700008B50120FEF7E6FA08BD000008B5114BD3
:101C80008022DA675200DA678022D200DA67802287
:101C90005201DA6780221201DA6780229200DA6745
:101CA000094A002313600121084A49421160084A89
:101CB0001360084A1360084B01221A60FFF7D8FF2F
:101CC00008BDC04604E100E00482044008820440EC
:101CD00004C000403CC0004000C0004008B5064BB6
:101CE0001A6801321A60054B1868FFF749FDFFF7C3
:101CF000C5FFC046C04608BD6403001020000010A8
:101D0000F7B5071C0C1C72B6FFF78EFF4F4B1A6815
:101D10004F4B1A60002F01D04E4B00E04E4B4F4A04
:101D2000042113604E4B4F4D1A680A431A6000237A
:101D30002B60A1071ED04C4B4C4A19680A401A6010
:101D400029684B4BA2070ED5EC2252010A432A60A8
:101D500080221A6052001A608022D2001A6080220B
:101D600052011A6003E0802212010A432A60802295
:101D700012011A60002F53D03E4B00241C603E4BD2
:101D80003E4E1C603E4B301C1C603E4B211C1C60B8
:101D9000FFF718FF201C0921221CFFF79DFE201CC5
:101DA0000921221CFFF7E8FE374B80211A683748CB
:101DB0000A431A6033680722934333603368022270
:101DC000134333600A21784302F018FE304B03229C
:101DD0001860304B1C60304B1A60304B304A196829
:101DE0000A401A601A6880210A431A60204A8B0050
:101DF00013601D4A1168194311602A6802211343B8
:101E00002B60284B01221A60274B1960274B194978
:101E10001A601C601A60186801221042FBD00A6028
:101E2000234B012252421A60224B1B68019362B677
:101E300030BFC0461F4B019A1B689A4205D11E4B0A
:101E40001868FFF79DFCFFF719FFF7BD38820440C3
:101E500034820440BF180000FF18000030820440A4
:101E600010ED00E004820440008204407FE2FFFFA6
:101E700000E100E004C00040040001406440044070
:101E8000044001400480014080800440841E000022
:101E900018C0004008C0004014C000403CC00040D2
:101EA0000FF0FFFF7880044070800440748004408D
:101EB00008820440640300102000001008B5FFF7FA
:101EC0001FFF08BD074B1A68013203D1064A11688B
:101ED000013111601A6801321A60044B1A6801322C
:101EE0001A6070477403001070030010680300103C
:101EF000074B98420AD8074A00231360064A013864
:101F00001060064A1360064B07221A607047C046ED
:101F1000FFFFFF007403001014E000E018E000E091
:101F200010E000E00B4A10B51368002800D1012032
:101F3000C1438B4208D91168994209D3591C1468CE
:101F400009188C42FAD3F6E71168C91A8142FBD30B
:101F500010BDC04674030010014B18687047C0469E
:101F600074030010064BFA211868064B10B589005F
:101F70001C6802F043FD044B5C43201810BDC046B2
:101F8000740300107003001037894100034B0122D5
:101F90001A60034B1A6801321A60704700C0004093
:101FA00078030010034B01221A60034B1A680132B8
:101FB0001A607047000001407C030010002803D124
:101FC000044B01221A6003E0012801D1024B186082
:101FD0007047C04604C0004004000140002802D100
:101FE000044B186004E0012802D1034B00221A6060
:101FF0007047C04604C0004004000140002801D1E1
:10200000044B02E0012804D1034B1A6802210A4361
:102010001A60704704C000400400014010B5002958
:1020200000D1134900280DD1124B80241A68224395
:102030001A60114B03221860104B1960104B1A6084
:10204000620211E0012811D10A4B80221868520067
:1020500002431A600B4B00221A600B4B03221960DB
:102060000A4B1A6080229202094B1A6010BDC046CA
:10207000FFFF0000808004407803001018C000407B
:1020800014C000407C0300101800014014000140FF
:1020900000E100E080231022DB051A60094B0822D2
:1020A0001A6000238022D2051268D10604D5064AA0
:1020B000934201D00133F5E7044898429B415842CE
:1020C0007047C04618000040FF0F0000FE0F0000E0
:1020D00008B58022154B1202DA67154B6C221A6084
:1020E000144B154A196800201140196019681960CD
:1020F000124B19680A401A601A6804211A600122FA
:10210000FFF7EAFC002004210122FFF735FD002043
:1021100005210122FFF7E0FC012200200521FFF745
:102120002BFD074B00221A6008BDC04604E100E009
:102130001800004030400440F8FCFFFF34400440E9
:1021400004800440F8B5174A174C0023236013603D
:10215000164A202113608022D20511602168144A9A
:10216000012903D0934203D00133F7E7934203D10F
:10217000FFF790FF002014E00E4F00253E68013E5F
:102180002368FF2B0CD83B689E4204D03E68FFF7C3
:10219000E3FE051C0A35FFF7DFFE8542F0D1E7E7D5
:1021A0002068F8BD8003001084030010880300102D
:1021B000FF0F00008C030010034B01221A60034B39
:1021C0001A6801321A607047004001409003001005
:1021D000174B70B501241C60164B1A6812191A604F
:1021E000154B1A68002A22D01A68144D013A1A6059
:1021F0001E68002E0DD02A68201C211CFFF7BCFC95
:102200002B68201CE31A2B602A680221FFF7B4FC1C
:102210000DE01B68201C2B602A68211CFFF7ACFC1A
:102220002A68201C0221FFF7A7FC054B1E6070BD29
:102230000080014098030010940300109C030010DC
:1022400004800140002803D1044B01221A6003E0FE
:10225000012801D1024B18607047C046044001407C
:1022600004800140002802D1044B186004E00128DA
:1022700002D1034B00221A607047C046044001405F
:1022800004800140002801D1044B02E0012804D160
:10229000034B1A6802210A431A6070470440014048
:1022A0000480014010B500280FD1124B80221C6819
:1022B000920022431A60104B032218600F4B1960E2
:1022C0000F4B1A608022D20211E0012811D1094B74
:1022D00080221868D20002431A600A4B00221A605A
:1022E000094B03221960094B1A6080221203084B24
:1022F0001A6010BD80800440900300101840014017
:1023000014400140980300101880014014800140DF
:1023100000E100E008B5184B1A680E231340062BA5
:102320000DD1164B9E221B68134205D0144ADBB216
:102330005360144B1B681EE0D9071CD501E0042B29
:1023400005D1104B1868C0B200F0B1F813E00C2BA7
:1023500006D10B4B8022596852000A435A600AE0AA
:10236000022B08D1054B1A68054B910601D50022B6
:1023700000E001229A6008BD0880004014800040FF
:10238000A00300100080004000487047A003001028
:10239000F7B52D4B2D4C8022002192030191061C94
:1023A000DA67201C902200F015FA019B0725A36034
:1023B000274B284F1A68AA431A6019680122114353
:1023C0001960254B1968A9431960196811431960F0
:1023D000224B80211868490101431960204B1A6083
:1023E00083223A601F4A126819681F4B18685043CD
:1023F00002F004FB311C000902F000FB1B4B102211
:102400001B491A60030A0B601A4BC0B20322186002
:102410003A60194A1560194A1D1C1068019010682D
:1024200060230340602BFAD110680123184202D0C8
:102430002B680193F8E723708022114B92031A60F6
:1024400005230B60F7BDC04604E100E0A0030010C7
:10245000A44004400C800040A84004408080044018
:102460009880044078800440840500102880004053
:10247000048000400080004008800040148000403C
:1024800000E100E008B5FFF77FFFC268031C1202FD
:10249000120E8218D07BDA681202120E0132D2B20A
:1024A0009A7352B2002A01DA00229A7308BD10B55D
:1024B000041CFFF769FFC2681204120E8218D4735D
:1024C000C2681204120E0132D2B2427352B2002A12
:1024D00001DA0022427310BD08B5FFF755FFC2684C
:1024E000C36812021B041B0E120ED01A431E984121
:1024F000C0B208BD70B500241D5D0619002D02D0C4
:1025000005550134F8E7121B301C131C002B03DDAA
:102510000170013B0130F9E7D043C0170240A01819
:1025200070BDF7B5051C01910093561E092B01D80B
:10253000041C0CE000980A2102F060FA0199031CC7
:10254000321C281CFFF7EDFF071C2C1807E0671B47
:10255000002E04DD019B013E23700134F7E7009853
:102560000A2102F08FFA3031781C2170FEBDF8B5D7
:102570000C1CD9175F18051C4F40561E092F12D985
:10258000381C0A21002B03DA02F038FA434202E039
:1025900002F034FA031C281C211C321CFFF7E7FF51
:1025A000041C2D1814E0002B00DA961E2A1CA91911
:1025B000891A002902DD14700132F8E7F443E417A8
:1025C00034402D19002B03DA2D232B7001340135F3
:1025D000381C0A2102F056FA30312970601CF8BD0F
:1025E000F7B5089F1E1C051C013A3B0901D1041CCC
:1025F00005E00093331CFFF7F3FF2C1806E0601B87
:10260000002A03DD2170013A0134F8E70F231F404F
:10261000092F01D8303704E0002E01D0373700E011
:10262000573727700130FEBDF0B585B0041C02910C
:1026300001D00021017000251178002906D1029FE8
:102640000023BD426CD22370281C6FE0029FBD4264
:10265000F5D2252902D00132217004E051782529D4
:1026600004D12170023201350134E5E7302902D06E
:10267000561C202100E0961C32782D3A50424241EF
:10268000B6180022307830277F423F18FFB2092F5A
:1026900007D80A277A438218D2B2303AD2B201362A
:1026A000F0E7AF18BC46029FBC4501D97A1BD2B2F5
:1026B000692818D00BD863282AD0642813D058284A
:1026C00032D11F1D1B68201C009301231DE07528BB
:1026D0000FD0782814D0732826D11F1D201C1B680A
:1026E000FFF708FF0AE01F1D201C1B68FFF73FFFD4
:1026F00004E01F1D201C1B68FFF713FF3B1C0BE0B1
:102700001F1D1B68201C00930023FFF769FFF5E7DE
:102710001868043320700120721C24182D188BE7D0
:10272000013C2370681E01E00120404205B0F0BD6D
:1027300010B50C1C131C6421221CFFF775FF10BD83
:1027400000B5031C9BB00A1C01A8191CFFF7F0FF81
:10275000632800DDFEE701A800F0B6F81BB000BD5D
:102760000FB407B504A908C9181C0191FFF7E8FFC9
:1027700003B008BC04B018470EB403B503AA08CAD6
:10278000191C0192FFF7D4FF02B008BC03B0184730
:1027900030B50C1C044303232340041C002B01D040
:1027A000002310E0032AFBD9CC58C4500433D41AB8
:1027B000032CF9D8131F9B0801339B00C418C918B8
:1027C00003231A40ECE7934203D0CD5CE554013378
:1027D000F9E730BD30B5031C840701D1032A01D8C5
:1027E0009A1814E00B060C041D1C25430D430C0223
:1027F0002543031C20C38418E41A032CFAD8131FA2
:102800009B0801339B000324C3182240E8E793424E
:1028100002D019700133FAE730BD021C031C981A6C
:102820000133591E09780029F9D17047031C0A7831
:102830001A70002A02D001310133F8E7704730B531
:102840000023934208D0C45CCD5C651B06D10133E4
:10285000002CF6D1201C02E0002000E0281C30BD36
:1028600010B50022835C8C5CA34204D10132002BA2
:10287000F8D1181C00E0181B10BD000008B5094B6A
:10288000FA211868890002F007F9FFF731FB96205A
:102890000002FFF77DFD0120FDF7D4FCFEF74EFF9F
:1028A00008BDC0468405001008B5FEF7CFFFFFF74E
:1028B00005F9FFF7ADF9FEF79FFBFEF78BFBFFF77E
:1028C000DDFFFFF7F3F808BD10B5041C20780028E1
:1028D00003D00134FDF706FDF8E710BD38B5051C3F
:1028E0000E24013C04D3295D0248FFF739FFF8E7C5
:1028F00038BDC0466056000038B51648FFF730FFB7
:10290000154C201CFFF7EAFF144D4221281CFFF74D
:1029100027FF201C0E30FFF7E1FF4321281CFFF7A3
:102920001FFF201C1C30FFF7D9FF0D48FFF718FFD1
:10293000201C2A30FFF7D2FF281C4E21FFF710FF82
:10294000201C3830FFF7CAFF616D0648FFF708FF0B
:1029500038BDC04663560000C0050010695600002F
:10296000705600007656000003110A2253430F22CE
:1029700010401818704738B50A21041C02F08CF872
:102980000A210501201C02F0DDF8281C084338BD8F
:1029900008B5C12252000E200221FEF73BFE024B79
:1029A00001225A7108BDC046B405001010B5084C8C
:1029B0006379002B01D1FFF7EBFF23790C221A4337
:1029C000A37901205B001A43011CFEF723FE10BD12
:1029D000B405001010B5074C2379002B08D163799A
:1029E000002B01D1FFF7D4FF01232371FFF7DEFF96
:1029F00010BDC046B405001008B5054B1A79002A71
:102A000005D000221A711A72DA70FFF7CFFF08BDE5
:102A1000B405001010B501210220FEF739FE064B67
:102A2000041C18787F231840FFF79EFF034B587053
:102A3000DC71201C10BDC04690050010B4050010CC
:102A4000014B01229A707047B4050010024B00221E
:102A50009A701A727047C046B405001008B5FFF7A7
:102A6000D9FF094B094A9978002908D0197A012918
:102A700001D8013103E010680549086000E01972CF
:102A80000021D970116008BDB40500106803001062
:102A90006C03001008B5FEF72FFE0C23184003D07E
:102AA000024B1A781043187008BDC046B4050010D8
:102AB00010B5FFF7EFFF054B1A781C1C530701D523
:102AC000FFF7CCFF0023237010BDC046B4050010F3
:102AD00008B50020FEF708FC002801D0FFF7E8FF4A
:102AE00008BD000010B5054C0023E371FFF7F0FFAF
:102AF000E379002B01D1FFF78DFF10BDB405001065
:102B000008B50948092102F029F8084BFA22D20039
:102B10001A80FFF7E7FF064B00221A60FA22054BE6
:102B200092001A6008BDC046B4050010BE05001032
:102B3000680300106C03001008B5FFF7C9FF002000
:102B400008BD08B5FFF758FF08BD000070B51D4C63
:102B5000061C637822781B021343A278A079120422
:102B60001343E2780D1C12061343174A13401A0A46
:102B7000237062701A0C1B0EE3706379A2702279C5
:102B80001B021343114A134023711B0A6371FFF7A1
:102B9000EBFE0F4B1B88C01830806079FFF7E4FE16
:102BA000B070E078FFF7E0FEF070A078FFF7DCFE91
:102BB00028706078FFF7D8FE68702078FFF7D4FEA1
:102BC000A87070BD900500107F7F3F3F071F000079
:102BD000BE050010F0B58DB0051CFEF769FD00289C
:102BE00004D1281C1249FFF7C7FD1EE00AAE0BAC4A
:102BF000211C301CFFF7AAFF3388F7780793B378BE
:102C0000267808936378A47809930A4B187900F022
:102C1000B7F8099B04900293009701960394281C2F
:102C20000549079A089BFFF7A7FD0DB0F0BDC04608
:102C3000825600009005001087560000F7B5048802
:102C40000E1C051C6421201C019201F01BFF114B7E
:102C50008FB2B078E41B1C80FFF78DFE0E4CA07085
:102C60007078FFF788FEE0703078FFF784FE2071FF
:102C7000E878FFF780FE019B6071A371A878FFF7E9
:102C80007AFEE071381CFFF776FE2072FEF722FD17
:102C9000FEBDC046BE050010A005001008B5021C10
:102CA000501E8241520100200121FEF7B3FC08BDF5
:102CB00038B5041C01200D1CFFF7F0FF201C00F0AC
:102CC00087F8072101F03EFF201C0A1C291CFFF792
:102CD000B5FF96204000FFF725F90020FFF7DEFF43
:102CE00038BD000073B5041CFFF794FE002801D125
:102CF00000203BE01E4B5D781E1C7378AB4207D171
:102D00000A20FFF70FF9FFF785FE0028F5D1EFE75E
:102D1000FEF7CEFC0028EBD001A96846FFF716FFAE
:102D2000684600F055F8051C01A800F031F8114B79
:102D300004199C420DD9E31701221343ED18281CF6
:102D4000694600F075F8002C01DA0B4B00E00B4BE4
:102D5000E418201C01A900F024F8281C072101F028
:102D6000F1FE68460A1C01A9FFF768FF76BDC04660
:102D7000B40500107F5101008051010080AEFEFFBC
:102D800007231840014B8000C0587047EC0000102A
:102D900002783C235A43417852185343827898185A
:102DA000704738B50C1C3C21051C01F0CBFE281CDB
:102DB000A1703C2101F070FE3C2101F0C3FE617066
:102DC000E121281C090101F067FE207038BD0000D8
:102DD00070B58378022100229942524104889621DD
:102DE0004901051C64180C20A41A42439B18033B9C
:102DF000992058430521023001F04EFE6E26FF3621
:102E000066436421A31086194942201CF61801F07C
:102E100043FEC82136184900201C01F03DFE034B3B
:102E20003018C018EB78C01870BDC046D382FFFFC1
:102E3000F8B5204B0C1CC5181F4B8000C0181F494B
:102E400001F02AFE03235843C617B60F3618B610F2
:102E5000AE19B600953E301C194901F073FECD172E
:102E6000AD0F6D180527AD107D430235281C992143
:102E700001F068FE081C391C01F00EFE0130E07004
:102E80009921281C01F008FE0C21023001F05AFEA5
:102E90004D1CEDB2A570301C094901F0FDFD094B38
:102EA0000C21C6180E20401B01F0F6FD36182680B6
:102EB000F8BDC04679050000652F0400B13A020054
:102EC000B505000094EDFFFFF8238A01DB001340F5
:102ED0004A05920E1343F8221202114019430A23A5
:102EE000594330B5CA1083181C1CEB345D78247824
:102EF000EA336C401B7824021C43835C201C58403E
:102F00000723194008418005800D30BD704700003F
:102F100008B5054B011E994201DD044BC118044858
:102F2000EA38FFF7D1FF08BDFF17000000F8FFFFE8
:102F3000135700000723594310B5084B59189C310B
:102F40000023CC5C0F2222400270CA5C01331209BC
:102F500042700230072BF4D110BDC046C0050010EE
:102F60000723594310B5074B59189C310023427869
:102F7000047812012243CA5401330230072BF6D1E0
:102F800010BDC046C005001070B5AD4C86B0E36EF4
:102F90006E465A1E934117363370AA4B9A6A191C13
:102FA000D006400F0138062807D801F013FD040CA5
:102FB0002012181A1D00022509E0636E16339B00CB
:102FC0001B591D1C15E0636E16339B00E55800234A
:102FD0000FE0A36DE56DAB420BDD0D2509E0022589
:102FE00003E00C25032304E00D252B1C01E00D2537
:102FF000EDE70D6150111F2800D91BE101F0F4FC31
:103000002000220029002C002F0033003B00440048
:1030100048004C00540061006E00760083008F0071
:103020009B00A800B800C500D500D300E100E40073
:10303000E700EF00FE0002010B010D010F01150179
:10304000E01801E0E0180E30EB1A591C01F086FD83
:10305000F0E0E0181C30F7E7211C0E3105E0E01825
:103060000E30E1180BE0211C1C31201C1A1C2B1CFB
:1030700001F0EDF8DEE0E018E1181C300E31EB1A3B
:103080005A1CFFF785FBD5E06F48011C0E31EDE7B8
:10309000E018011C1C31F2E7226E1021002A00D03A
:1030A0000A21221C0E3206E0226E1021002A00D0D6
:1030B0000A21221C1C32029100950196201C211C21
:1030C00053E0216E012232701022002900D00A2222
:1030D000009501960292201C211C45E0226E1021D1
:1030E000002A00D00A21221C0E3213E0216E012298
:1030F00032701022002900D00A2200950196029217
:10310000201C211C4DE0226E1021002A00D00A2133
:10311000221C1C32009501960291201C6AE0226E4E
:103120001021002A00D00A21484A029100950196F8
:10313000101C111C19E0216E1020002900D00A205B
:10314000424A0290111C1C3900950196101C0CE09B
:10315000216E012232701022002900D00A223B4940
:10316000009501960292081C002201F07AF861E0B5
:10317000226E1020002A00D00A20344A0290111C2E
:103180001C3900950196101C35E0216E0122327029
:103190001022002900D00A222C49009501960292A3
:1031A000081C002227E001223270226E1021002A22
:1031B00000D00A21254A029100950196101C002199
:1031C00019E0009620481BE00096204818E0226E87
:1031D0001021002A00D00A21221C1C3206E0226E97
:1031E0001021002A00D00A21221C0E3200950196DF
:1031F00002910020211C01F05CF81BE00096201CCD
:10320000002103E0211C1C310096201C1A1C2B1CE1
:1032100001F0ACF80EE0201C02E00B4800E00B4887
:10322000191C2A1C01F0B9F804E0201C191C2A1CE6
:1032300001F0BDF833780120E36606B070BDC046EA
:10324000C00500105C0D0010CE050010DC0500105C
:10325000064910B50A1C883213681C1C1E34A400D1
:103260006050013303210B40136010BDC0050010F6
:10327000054B0322191C88310868013802400A6096
:103280001E329200D0587047C0050010F7B5124F9B
:103290003D1C8C3528680130FFF73AFE0F4EBB6E9F
:1032A000B26A041C01920122F06202409A4210D1DB
:1032B000830703D428680230FFF7CAFFFF239B006F
:1032C000019A1C40A40193101C438C3701233C60DD
:1032D000F3600220FEBDC046C00500105C0D00106A
:1032E0000C490D488A6A031C8C3370B51D68D305E0
:1032F0009B0E0C1C910500D5403B866E921001215F
:103300000A40B24203D18C30EB180360E160012027
:1033100070BDC0465C0D0010C005001008B5084B1C
:103320005A1CD07F9A1CD27F000112021043033333
:103330001A7FDB7F10431B031843FFF789FF08BD8B
:10334000C005001008B5FFF793FF0323044A0F21BF
:103350009A180140013311770011072BF6D108BDEF
:10336000C005001008B5FFF783FF034B01228C3323
:103370001860024BDA6008BDC00500105C0D00103B
:1033800010B5064CA36E002B06D0FFF771FF044B5F
:103390008C3401222060DA6010BDC046C0050010E8
:1033A0005C0D001010B5064CA36E002B06D1FFF784
:1033B0005FFF044B8C3401222060DA6010BDC046F0
:1033C000C00500105C0D001008B5104B0022596AB2
:1033D0001A62914214D05969914216DD012906D131
:1033E000D969914203D0DA610A2299615A615A6916
:1033F000032A02DD06490120C866013A5A6104E049
:10340000044B1B68002B00D0984708BD5C0D0010D2
:10341000C005001030040010074B5A6A002A02D081
:103420005A69002A07DD9A690F21044B1140D977A8
:1034300012110133DA7770475C0D0010C0050010DF
:10344000044B597F9A7F090112020A43197F0A43EC
:103450005A677047C00500100B1C093B10B5012BC3
:103460000FD80023074A9A18147FC25C944205D0F3
:10347000054B08395A681143596002E001330E2B9D
:10348000F0D110BDC00500105C0D001008B5082972
:103490000DD0192913D1427808231A4202D00022F4
:1034A000027002E00F2303700723437005E000233E
:1034B0000022C25401330E2BFAD1FFF751FD08BD93
:1034C00030B5114D85B06C6F002802D00F239C439E
:1034D00004436C67FF2C05DD281C1C300E2101F015
:1034E0003DFB0FE06846211CFFF724FD6846211CC8
:1034F000FFF7CCFF00236846C15CEA18013311775F
:103500000E2BF8D105B030BDC0050010134B30B5FF
:10351000596F0F229143041C0C4385B05C671D1C3E
:10352000082C19D0FF2C17DC6846211CFFF702FD80
:103530006846211CFFF790FF0023EA18127F6946B6
:10354000CA5401330E2BF8D16846211CFFF79EFFA9
:103550006846211CFFF704FD05B030BDC005001012
:103560001FB50F4C616F082918D0FF2916DC68467B
:10357000FFF7E0FC6846616FFFF76EFF0023E2187B
:10358000127F6946CA5401330E2BF8D16846616F29
:10359000FFF77CFF616F6846FFF7E2FC1FBDC04686
:1035A000C005001010B50D4C631CD87FA31CDB7F39
:1035B00000011B021843E37F1843E31CDB7F1B035E
:1035C0001843FFF7A5FC0F23021C1A4022770211B3
:1035D000134000126377A07710BDC046C0050010ED
:1035E000044B5A6E16329200D258121A51424A4176
:1035F000DA667047C0050010044B5A6E163292000E
:10360000D158013900D50D21D1507047C0050010A7
:10361000054B5A6E16329200D15801310E2900D155
:103620000021D1507047C046C0050010094B5A6EAA
:1036300016329200D2580D2A03D11A1C2932127860
:1036400005E09A18507F117F0001021C0A435A6559
:103650007047C046C0050010084B10B55A6E0F24C5
:1036600016329200D1585A6D58181440013104771F
:103670000D2902DC5B1812111A7710BDC00500106D
:103680000E4B30B55A6E596D16329200D2580D2A33
:1036900007D11C1C2934F0202478084020435865A9
:1036A00007E09818447F057F24012C435C650C11CA
:1036B00044779B180F221140197730BDC0050010C8
:1036C00008B503480E22011C1C39FFF761F808BD3C
:1036D000F805001008B503480E22011C1C31FFF745
:1036E00057F808BDDC05001008B504480022011C8D
:1036F0001C310D2300F0ABFD08BDC046DC050010F9
:1037000008B503480E22011C0E39FFF741F808BD29
:10371000EA05001008B503480E22011C0E31FFF720
:1037200037F808BDDC05001008B504480022011C6C
:103730000E310D2300F08BFD08BDC046DC050010E6
:103740000023044A00219A18463201331170082BD5
:10375000F7D17047C0050010C31C421E00209342E1
:1037600007D004494000591846310978013B084305
:10377000F5E77047C005001010B50B1D994208D041
:10378000044A01248A180440463214704010013162
:10379000F4E710BDC005001038B50020FFF7DCFFCE
:1037A000084C051C0021207FFFF7E6FF0420257749
:1037B000FFF7D2FF0421051C607FFFF7DDFF65776F
:1037C00038BDC046C005001010B50020FFF7C4FF8B
:1037D000034C20770420FFF7BFFF607710BDC04681
:1037E000C005001010B5054C0021207FFFF7C4FF75
:1037F000607F0421FFF7C0FF10BDC046C005001068
:1038000010B5094C231C8C3318680130FFF780FB7E
:10381000064B021CD8620F231A4022770211134074
:1038200000126377A07710BDC00500105C0D00107A
:1038300010B5084C0E21201C01F090F9201C0E3010
:103840000E2101F08BF9201C1C300E2101F086F9AD
:1038500010BDC046C005001010B50C4B191C0E3130
:103860001A1C187F1C7801332043D8768B42F8D17C
:10387000936E002B08D0064B1B690D2B04D1137FD0
:10388000111C29310B70537310BDC046C0050010C8
:103890005C0D001010B50C4B191C0E311A1C1C7F4E
:1038A000187801332040D8768B42F8D1936E002BE4
:1038B00008D0064B1B690D2B04D1137F111C293135
:1038C0000B70537310BDC046C00500105C0D001096
:1038D00030B5002185B00E4B421C1818007F6C4695
:1038E00008550D25D40F181C002395425C416442F5
:1038F000013122400E2901D0101CECE76C46E15C3E
:10390000C218013311770E2BF8D105B030BDC04677
:10391000C0050010074B10B55A6E16329200D458ED
:10392000611E1C19D1502077002901DA0D21D150D8
:1039300010BDC046C0050010034A0023111C94317D
:1039400098320B6013607047C0050010034B0122D2
:10395000943319684A401A607047C046C005001089
:10396000044A002313678C321360034B0122DA6090
:103970007047C046C00500105C0D001010B59E4C8D
:103980000F20A16A9D4A8B101840891101385256A8
:103990000E2848D801F01EF8080F171F23472947A3
:1039A0004731474747353900002A3CDB944B9A188A
:1039B0004032002305E0002A35DB914B9A18403253
:1039C000012393712DE0002A2DDB8D4B9A18403294
:1039D0009279DA6625E0081CFFF79CFF21E0002AB7
:1039E00021DB101CFFF7FCFD1BE0002A1BDB844BD6
:1039F000596E16318900CA5013E0081CFFF786FD86
:103A00000FE0081CFFF75CFD0BE0002A0BDB101C2D
:103A1000FFF75EFF05E00C2B23DD162B28D1FFF707
:103A200005FE0120EEE0982B03D1754B00221A66AB
:103A3000F7E7982B6CDC382B03D1714B01205866CB
:103A4000E0E0382B30DC1C2B02D1FFF739FEE8E731
:103A50001C2B12DC0C2BDED1694B01209833186033
:103A6000D0E00120002B00D1CCE001204042C9E091
:103A7000182BFAD1FFF774FFD3E7282B03D1604B43
:103A800000225A66CDE7282B04DC262BEDD1FFF768
:103A9000E3FDC6E72C2B02D1FFF71CFEC1E7362B56
:103AA000E3D1FFF7EDFDBCE7662B02D1FFF732FE55
:103AB000B7E7662B16DC4C2B03D1FFF7A1FE0220E3
:103AC000A0E04C2B04DC3C2BCFD1FFF70DFEA8E788
:103AD000562B02D1FFF714FEA3E75C2BC5D1FFF7ED
:103AE0001DFC9EE76C2B02D1FFF72CFC99E76C2B99
:103AF00004DC682BB9D1FFF79BFE92E7762B02D14D
:103B0000FFF712FE8DE7882BAFD1FFF785FC88E722
:103B1000E62B02D1FFF758FE83E7E62B35DCC82BF6
:103B200002D1FFF713FF7CE7C82B16DCA82B03D1CB
:103B3000334B0120186665E0A82B04DC9C2B94D144
:103B4000FFF77EFC6DE7B82B02D1FFF7F5FE68E7C3
:103B5000BC2B8AD1FFF704FD63E7D62B02D1FFF718
:103B600041FE5EE7D62B05DCCC2B00D07DE7FFF7CE
:103B700019FD56E7D82B02D1FFF702FC51E7DC2BE9
:103B800000D072E7FFF768FE4BE7F32B02D1FFF797
:103B90001BFC46E7F32B17DCEC2B02D1FFF77AFE78
:103BA0003FE7EC2B05DCE82B00D05EE7FFF7FAFBE4
:103BB00037E7F12B02D1FFF7C3FD32E7F22B00D03C
:103BC00053E7012020621DE0F62B02D1FFF7E4FD50
:103BD00027E7F62B05DCF52B00D046E7FFF70CFDB9
:103BE0001FE7F72B02D1FFF713FD1AE7F82B00D0E0
:103BF0003BE7FFF7B7FB14E75C0D001013930000E1
:103C0000C005001010BDC04638B5184C231C8C33BD
:103C10001868FFF77DF9164B0022E16EDA60E26664
:103C200003229862A16610401D1C022809D0904210
:103C30000AD0012802D0FFF7A1FE07E0FFF726FB1C
:103C400004E0FFF7A1F901E0FFF74AFB00280BDDD4
:103C5000EB68002B04D1231C8C3319680A181A60F6
:103C6000903422681318236038BDC046C005001088
:103C70005C0D0010034B0122DA660F229A775A7707
:103C80001A777047C005001010B5054C0549201C77
:103C900000F064FFFFF7EEFF0123636610BDC0462E
:103CA000C00500109C0700007047000030B50C4DA7
:103CB000049C28600B4801600B490A600B4A1360A2
:103CC0000B4B039A1A600B4B0B4A1C600B4B1C608E
:103CD0000B4B1A600B4B0C4A13600C4A136030BD3F
:103CE0005404001060040010680400103C0400102C
:103CF0003404001010010010513D00005C0D001054
:103D000030040010A93C0000640400104C040010B2
:103D1000014B18607047C04638040010094B10B5BD
:103D20001A68191C084B002A03D1084C2468226029
:103D300003E01A68904200DA101C186001230B603F
:103D400010BDC046400400105C0400103804001090
:103D500013B5002300930193114B124C1A68124BB8
:103D600011681868814202D12268009208E0126846
:103D70001A600E4B1B68002B02D0684601A99847B9
:103D8000009B2360002B04D0094A64209361FFF755
:103D9000C5FF009A531E9A41064BDA6613BDC04612
:103DA0003C040010500400100C01001060040010CE
:103DB0005C0D0010C0050010034B1B68002B01D1E7
:103DC000024A13607047C0464804001040040010C7
:103DD000014B4A3318787047C005001038B5164BB0
:103DE0001A1C98321268002A04D0144B1C68012354
:103DF0001C4001E094331C68114DAB689C4202D119
:103E00006A68002A16D0002C02D1002B0AD111E0DA
:103E10000C4B1B68002B02D0201C696898470023BC
:103E20006B6006E0074B1B68002B02D0201C211C96
:103E30009847AC6038BDC046C0050010440400106F
:103E40005C0D00105404001008B5084A084B1268B5
:103E500019688A1A05D5FA2252001A60054B1A68A9
:103E600001321A60FFF7BAFF08BDC04634040010E3
:103E70001401001044040010F8B50E1C0E21041C9F
:103E8000171C00F06BFE174B03259E4211DD092322
:103E900063730123237323E0301C0A2100F052FED8
:103EA000301C61550A2100F0F7FD0135061C0D2D6F
:103EB00001D0002EF0D1EF1B033F27706B1E022BA9
:103EC00005D0E15C621BD2185173013BF7E70F2369
:103ED0005D1B013D6B1C032B02DD00236355F8E7DE
:103EE000F8BDC046FFC99A3B37B5041C0025002326
:103EF00000930193124B1B68002B02D0684601A966
:103F0000984700980135002800D000250220FCF7D2
:103F100016FA0C4B1A680C4B1168186881420AD0CB
:103F200012681A60FFF790FF002C04D0013C002CAF
:103F300001D1201C02E0032DD9DD01203EBDC04689
:103F4000600400103C04001058040010F7B59B23D7
:103F50001E4A5B000D1CD45C38213023FF33FF3137
:103F6000D35C515C161C002C02D00F22114002E0E1
:103F70008024072164009A225200B75C3622FF3267
:103F8000B25CE31ABA1A80277F003C1B0094072416
:103F9000611A019101320E490024FEF7EDFB2C70ED
:103FA000281CFEF73AFC34273119FF37CB1935317D
:103FB000FF311F780B784122121B2818FB1A054984
:103FC000013CFEF7D9FB631DEAD1F7BDC005001027
:103FD0002393000030930000F0B5544D544C2B1C3B
:103FE00094331B6893B0061CA061E161002B17D1CC
:103FF00018280BD1C32909D14E4B1B680F2B05D1B3
:10400000281C38300E21162200F00CF9A06918285F
:1040100004D1E269332A01D100F0AAF8FFF72AFEA1
:10402000002E02D00A23636100E06661424BA06962
:10403000424F18603B68424E1B683360FFF7BCFE7E
:10404000012300222B6701923E4B1B68002B1AD0E4
:104050003D4E3368371C002B15D01B68002B04D154
:104060003A4B1B6898473B68F7E733681A68013A90
:104070001A60374A1368002B05DD013B1360002BE3
:1040800001D1FFF799FEFFF7BFFD002801DAFCF729
:1040900005FA019A40239A432E4B9A4208D1A26A0C
:1040A00010239A432C4B9A4202D10A20FFF736FE86
:1040B000A36A2E1C8C360193284A3368934203D09E
:1040C000274A93420BD019E0FFF788FEFCF766F908
:1040D0001B481B4A0068031C013B13600EE0214F84
:1040E0003B68002B0AD002A80AA9FFF72FFF3B6804
:1040F00002A80AA998473368273333601A4B1B6814
:1041000098470E48194B026818681168814206D01A
:1041100012681A60FFF798FE0C4B1B6898472A6FCD
:10412000002A91D1FFF75AFE13B0F0BDC005001070
:104130005C0D001010010010500400103C04001031
:104140000C0100104004001038040010640400103A
:104150005C04001026020000EB030000790D000053
:104160003E270000680400104C04001058040010A2
:10417000F7B5274E002033681C68FFF7B5FE33689B
:104180001A689442FCD01B6801272D33FF3301933A
:10419000FFF770FD1F4C0A231F4D63611823A361B5
:1041A0001523E3612B1C9033002267621A60FFF72E
:1041B00061FD2F673368019A1B689A420CD0FFF7A4
:1041C00023FD3268154B116818688142F2D01268DD
:1041D0001A60FFF739FEEDE72B1C012790331820FA
:1041E00000211E686762FFF7F7FE0D4B301C19684F
:1041F00000F052FC3835011C0422281CFFF73CFE5D
:104200001823A3610023301C6762E361FEBDC04632
:104210003C0400105C0D0010C00500105804001094
:104220003404001070B5002A10DD047801231C400E
:104230004B1E002B08DBC55CE4006E083443C454FD
:104240000124013B2C40F4E7013AECE770BD30B5A6
:104250009A4205DC845C8D5C85548C540132F7E70E
:1042600030BDF0B5069E051C07A804783078002AFA
:1042700017D0059EB34217DCCE5CD75CF7193F1808
:104280000020A74201DB3F1B0120EF540133F0E780
:10429000CA5C12180020A24201DB121B0120EA5462
:1042A0000133059A9342F3DD01231840069B1870F1
:1042B000F0BDF7B50AAC2478099D0094089E2C78CF
:1042C00000282DD0002928D0002A18D0B34248DC7D
:1042D000CF5CD55C7F1B3F1B0024A74202DA009C09
:1042E0003F190124C7540133F0E7CA5C121B0024B4
:1042F000551C02D1009A0124013AC2540133B34241
:10430000F3DD2EE0D15C4942091B0024A14202D01A
:10431000009F0124C919C1540133B342F2DD20E0EA
:10432000002914D0002A08D0B3421ADCCD5CD05C3E
:104330000133281A041BE40FF6E7B34211DCCA5C10
:104340000133141B013462425441E4B2F5E7B34235
:1043500007DCD15C013349420C1B611E8C41E4B285
:10436000F5E701231C40099B1C70F7BD70B5049C48
:104370000125257000290BD09A420BDC865C8D5CF0
:10438000AE4209D10132F7E7815C002904D1013244
:104390009A42F9DD0023237070BD914204DA43187C
:1043A0005B7843540131F8E70023435470478A4255
:1043B00005DD8318013B1B788354013AF7E700239E
:1043C00083547047F7B5134A134C13785278C35C83
:1043D000134000D040231149236012310091002284
:1043E0000023A6187360009B0125123B1F785978A3
:1043F000C75D394202D077682F437760009F023350
:104400006D00BB42F2D1123304320093282AE7D167
:104410000020FEBD0D0200101C0F001059010010FD
:10442000122330B54B43334A0131D318052251438F
:104430001A785C78825C144204D02F4A5F245218A8
:10444000947054709A78DC78825C144204D02A4AC2
:104450007C245218533214701A795C79825C1442AD
:1044600004D0254A7C245218A33214709A79DC793E
:10447000825C144207D0204C5F226418251CA235B0
:10448000A1342A7022701A7A5C7A825C144204D0B9
:10449000194A7C245218A03214709A7ADC7A825C11
:1044A000144204D0144A7C245218503214701A7BDF
:1044B0005C7B825C144207D00F4C5F226418251C81
:1044C000523551342A7022709A7BDC7B825C144214
:1044D00004D0094A2E245218A43214701A7C5B7C32
:1044E000825C134204D0044B5918F43127230B701B
:1044F000002030BD590100108C0D0010F8B52E4D74
:10450000061C00272C1C281C20214F22FEF762F9D4
:10451000002F04D02A1C7C2339322B7013702B1CE3
:104520004F33002201371A705035052FEBD1211C73
:104530002D2338310B70211C37310B70A121A37052
:10454000637049005F2363544221FF316354A32108
:1045500049006254194A11785278715C0A4204D0B9
:10456000221C53325234137023700024211C301C3F
:104570000134FFF755FF0A2CF8D10024104B114DE0
:10458000E25C1B19B15C58780F4A6300084201D005
:10459000D15805E0D058FEF740F90C49091A0A3104
:1045A000281C023400F0E4FA122CE7D1281C084938
:1045B00000F0DEFA0520F8BD8C0D00100D02001091
:1045C00018010010CC0E00102C0100100F0200107A
:1045D00038930000F0B585B00190FCF7FBFCA24CCD
:1045E000A24F00260C257543002E00D10125A04BBB
:1045F0001B68012B02D0022B10D001E09B4F0EE074
:10460000002B0CD12168C90700D4ACE0681CC0B2F3
:10461000002107220223FCF755FDA4E0954F00235B
:1046200003A8437023687F2213405C2B00D191E0E4
:1046300027DC382B00D187E011DC072B65D005DCA7
:10464000022B00D18DE0062B40D0DBE7212B00D1DF
:104650007EE0232B00D181E01C2BD3D17CE04F2BBB
:104660004DD007DC3F2B61D0402B61D0392BC9D115
:10467000432374E0542B71D05B2B3ED0502BC1D11F
:1046800066E0732B62D00FDC662B3AD004DC5E2B25
:1046900052D0622B60D0B5E76F2B3AD0712B4FD040
:1046A0006D2BAFD135235AE0792B47D006DC762B22
:1046B00048D0772B3ED0742BA4D143E07D2B22D061
:1046C0007F2B24D07C2B9DD1422348E031230370E3
:1046D000022E00DCDCE0231C083B1B681A40542A35
:1046E00032D0032E00D1D3E0231C0C3B1A687F2369
:1046F0001340542B00D0CBE026E032232FE03323AD
:104700002DE034232BE0362329E0372327E038231C
:1047100025E039230370062E00DCB9E0231F1B6857
:104720001A404723232A00D0B2E018E0302316E0D5
:104730002D2314E0412312E0442310E045230EE032
:1047400046230CE048230AE04C2308E0502306E00F
:10475000522304E04F2302E0552300E04E23037070
:1047600096E04923FBE721680222114205D0A81DEB
:10477000C0B200210623FCF7A5FC236804210B42EC
:1047800005D0A81DC0B202220623FCF79BFC2368BB
:1047900008210B4205D0681CC0B207220223FCF797
:1047A00091FC2168C90606D5681CC0B2042102220A
:1047B0000623FCF787FC23689B0606D5681CC0B25D
:1047C000002102220623FCF77DFC2168490606D55C
:1047D000681CC0B2042107220223FCF773FC236883
:1047E0001B0607D5281C09300222C0B20821131C61
:1047F000FCF768FC2168C9050BD5EDB2281C09300F
:10480000C0B20B210A35FCF749FCE8B20A21FCF7DB
:1048100045FC013604340B2E00D0E3E6164B1B6832
:10482000002B05D0154800210922154BFCF7C0FCD0
:10483000144D00240235AB1E1A7801996B1E8A5C58
:104840001B78134208D0104BA200D0580F4B0922FE
:10485000E15C0B4BFCF7ACFC01340235092CEAD1CE
:10486000FCF7C2FB05B0F0BD1C0F001008000010E3
:104870001C020010000000104C02001042930000C7
:104880001400001018010010200200105001001048
:104890003B1C291C0022FCF78BFC23681B0605D55A
:1048A000E91D074800223B1CFCF782FC2368DB055E
:1048B000AFD5E91D034800223B1CFCF779FCA8E7B3
:1048C0008D5500004093000038B5FFF781FA0624AB
:1048D000002805D1FCF788FB38BD01340E2CF9DC2B
:1048E0000321201C00F0D8F80321C5B2201C00F0E1
:1048F00029F9281CC9B2FCF7D1FB092CEDD10B24F6
:10490000EEE7000038B5041CFFF75CFD201CFFF744
:1049100061FE094B1B78002B0DD0201CFFF7EEFD2C
:10492000064CC8235B00E518211C05485034FDF7F0
:1049300017FFAC42F8D138BD740400108C0D001084
:10494000CC4C000000B589B000280ED0FCF70DFB60
:1049500001A80921FEF7EEFA684612300A21FEF797
:10496000E9FA01A8FFF7CEFF08E0FCF706FB044BCD
:104970001B78002B02D00348FDF7F2FE09B000BD02
:104980007404001044930000FEE7FEE708B500231E
:104990000B4A0C499A188A4204D20B49C95C01336C
:1049A0001170F5E7094B0A4A591C013B934203D2A7
:1049B00000221A700B1CF6E7FBF7A0FFFEE7C046CB
:1049C00000000010440200109B93000045020010FC
:1049D000480F001002B4714649084900095C4900BB
:1049E0008E4402BC7047C04603B47146490840007B
:1049F0004900095A49008E4403BC7047002934D04D
:104A00000123002210B488422CD301242407A142A0
:104A100004D2814202D209011B01F8E7E400A1425D
:104A200004D2814202D249005B00F8E7884201D3F8
:104A3000401A1A434C08A04202D3001B5C082243D0
:104A40008C08A04202D3001B9C082243CC08A04241
:104A500002D3001BDC082243002803D01B0901D02D
:104A60000909E3E7101C10BC7047002801D00020A2
:104A7000C04307B4024802A14018029003BDC046DB
:104A8000D90000000029F0D003B5FFF7B9FF0EBC34
:104A90004243891A1847C046002941D010B4041C6B
:104AA0004C40A44601230022002900D54942002899
:104AB00000D5404288422CD301242407A14204D2CD
:104AC000814202D209011B01F8E7E400A14204D2AD
:104AD000814202D249005B00F8E7884201D3401AC4
:104AE0001A434C08A04202D3001B5C0822438C08E6
:104AF000A04202D3001B9C082243CC08A04202D350
:104B0000001BDC082243002803D01B0901D009093F
:104B1000E3E7101C6446002C00D5404210BC7047EF
:104B2000002806D003DB0020C043400801E08020BD
:104B3000000607B4024802A14018029003BDC04617
:104B4000190000000029EBD003B5FFF7A7FF0EBC4A
:104B50004243891A1847C0467047C046421800238E
:104B6000002903D0037001309042FBD17047C0464A
:104B700070B5061CB30717D133680F480F4D1A18CC
:104B80009A43301C2A420FD1043002680A4BD418D1
:104B900094432C4208D104300268074BD418944344
:104BA0002C42F1D000E001300278002AFBD1FDF761
:104BB0003DFE301C70BDC046FFFEFEFE8080808042
:104BC00025732025730D0A00444D3135005345529D
:104BD00049414C20434F4E534F4C45007265616430
:104BE00079000D0A4279652E2E2E0D0A004E4F00D7
:104BF000203F002573202573202025694D485A0049
:104C000056323200202025692E2530336956002087
:104C100025735254432000444D343100444D343107
:104C2000204F4B0020204552523A20256900424136
:104C300044204B4559202530327800202D20253046
:104C40003278004C43443A25303269202D202569C2
:104C500000505245535320454E54455220544F2046
:104C6000534156450025633120484F555200747515
:104C7000726E6564206F6E003C52455345543E0D84
:104C80000A00426164206E756D6265722E0D0A0025
:104C90004241543A2025696D560D0A000D0A25300F
:104CA000327820200057616974696E6720666F72E0
:104CB00020646174612E2E2E0D0A00426164206D05
:104CC0006F64656C0D0A00526561642025730D0ADE
:104CD000004641494C4544006F6666004C43442001
:104CE00064656275672025730D0A00436F6E736FEC
:104CF0006C652074696D656F7574207365742074BC
:104D00006F202569206D696E757465730D0A00004A
:104D10000000005C000C000C7C287C7C447C24108F
:104D200048285408000C003844004438002010087B
:104D3000103810804000101010004000201008387B
:104D40004438007C006454484454281C107C4C5463
:104D50002438542004740C28542808543800500077
:104D6000805000102844282828442810045408386B
:104D70004C5C7814787C54283844447C44387C5407
:104D8000447C14043844347C107C007C0020403C7B
:104D90007C106C7C40407C087C7C047C7C447C7C6B
:104DA00014083844787C1468485424047C047C40FB
:104DB0007C3C403C7C207C6C106C1C601C64544C23
:104DC0007C4400081020447C000804088080800493
:104DD00008007844780007080400000000BF01BF05
:104DE000010905000007000700070007130A00007B
:104DF0002000E400FC003F00E700FC003F0027002B
:104E0000040F0800000C011E01FF03FF032201E252
:104E100001C2190D00000E001F0011019101FF00D9
:104E20007E00FC00FE0113011101F001E0140A00F4
:104E300000EE00FF0111011101BF01EE00E00130A1
:104E4000011001050300000F000F0A050000F80023
:104E5000FE03070701040B0600000000010407071A
:104E6000FE03F80F08000000000A000E001F001FDC
:104E7000000E000A11090000100010001000FE00D2
:104E8000FE001000100010080400000004800780DD
:104E9000030D07000010001000100010001000109B
:104EA000080400000000800180010D07000C000FC5
:104EB000C003F0003C000F00030F080000FE00FFDD
:104EC00001010101010101FF01FE100800000000C5
:104ED00002010201FF01FF010001000110080000B2
:104EE0008601C7016101210131011F010E010F0877
:104EF000000082008301110111011101FF01EE1177
:104F0000090000300038002C002600FF01FF0120BE
:104F100000200F08000080009F011F0111011101F6
:104F2000F101E10F080000FC00FE010B010901097D
:104F300001F901F00F08000001000100C101F101B9
:104F40003D000F00030F080000EE00FF01110111EA
:104F5000011101FF01EE0F0800001E003F012101B9
:104F60002101A101FF007E0804000000008C018CDB
:104F7000010804000000048C078C031209000020C3
:104F80000070005000D80088008C01040104011159
:104F90000900004800480048004800480048004810
:104FA000004811090000040104018C018800D800A8
:104FB00050007000200D07000002000300B101B98D
:104FC000010F0006190D0000F800FC010603FB06A6
:104FD000FD0505050505FD05FF050601FC01F812A7
:104FE0000900008001F0017C004F004F007C00F0C0
:104FF0000180010F080000FF01FF01110111011FD5
:1050000001FE01E0110900007C00FE0083010101A6
:105010000101010183018211090000FF01FF01016B
:1050200001010101018301FE007C10080000FF0165
:10503000FF01110111011101110111010F080000FF
:10504000FF01FF0111001100110011000112090000
:10505000007C00FE008301010121012101E301E246
:105060000112090000FF01FF0110001000100010E4
:1050700000FF01FF010A0500000101FF01FF01011E
:10508000010B060001000101010101FF01FF1008F1
:105090000000FF01FF0138006C00C6008301010120
:1050A00010080000FF01FF010001000100010001E4
:1050B0000001160B0000FF01FF010F003C00F00093
:1050C000F0003C000F00FF01FF0112090000FF018A
:1050D000FF010F001C007000E001FF01FF01130A37
:1050E00000007C00FE008301010101010101830138
:1050F000FE007C0F080000FF01FF012100210021BC
:10510000003F001E140A00007C00FE008301010124
:10511000010101038307FE047C0412090000FF0162
:10512000FF01210021007100DF008E010001110943
:1051300000008E009F011101110111011101F30105
:10514000E211090000010001000100FF01FF01015F
:1051500000010001110900007F00FF008001000133
:1051600000018001FF007F1109000007001F007887
:1051700000E001E00178001F0007190D00000F009A
:105180007F00F001E0017C001F001F007C00E001B7
:10519000F0017F000F120900008301C7016C003885
:1051A0000038006C00C701830111090000010007ED
:1051B000001E00F801F8011E00070001120900009E
:1051C0008101C1016101310119010D0107010301D3
:1051D0000004040200007F01090500000700000030
:1051E0000000070B064400FF0144004400FF014497
:1051F0000B0600008C001201FF032201C40D078280
:105200000045002500920048014401820C06000080
:10521000E60019012601C00020010704000000007B
:10522000010002080400000000FE01010208040061
:105230000000000102FE010B060000880050002063
:10524000005000880B06000020002000F80020001D
:105250002006030000000400020B060000200020CE
:1052600000200020002006030000000000010905C6
:105270000000800160001800060B060000FE00011F
:105280000101010101FE0804000002000200FF010B
:105290000C06000082014101210111010E010B06E3
:1052A00000008200010111011101EE0B06000060F7
:1052B0000058004600FF01400B0600009F00090156
:1052C00009010901F10B060000FE00110111011195
:1052D00001E20B0600000100C10131000D00030BCB
:1052E000060000EE00110111011101EE0B06000095
:1052F0008E00110111011101FE0804000000008C54
:10530000018C01080400000000000208010A0500E9
:105310000020005000880004010B060000500050DF
:1053200000500050005009050000040188005000A2
:10533000200B06000002000100610111000E0D07A4
:105340007800860132014902390242027C0E078050
:105350000170004C0043004C00700080010B0600FF
:1053600000FF01110111011101EE0B06FE00010108
:10537000010101010101820B06FF0101010101018F
:105380000182007C0C060000FF01110111011101D6
:1053900001010B060000FF01110011001100010CBA
:1053A00006FE000101010111019100F2010C06FF4E
:1053B000011000100010001000FF010804000000A0
:1053C000000000FF010704C00000010001FF0E07FC
:1053D0000000FF01180024004200810000010C06BB
:1053E0000000FF0100010001000100010E07FF01A4
:1053F0000C003000C00030000C00FF010C06FF0163
:10540000060018002000C000FF010B06FE0001018D
:10541000010101010101FE0B06FF01110011001144
:105420000011000E0C06FE00010101014101810185
:10543000FE020C06FF011100110011002900C60137
:105440000B0600008E00110111011101E20B060094
:105450000001000100FF010100010B06FF00000137
:10546000000100010001FF0D0703001C0060008027
:105470000160001C00030D071F00600080017C001C
:10548000800160001F0E07830144002800100028DF
:1054900000440083010D07030004000800F0010828
:1054A000000400030E0781014101210111010901DE
:1054B0000501030100070008000A0100181110137C
:1054C0003831303378717073C8C1C0C3888180832C
:1054D00084848782C5C4C7C2757477723534373205
:1054E0001514171202070208020100030109030440
:1054F00002040205030500062024282C383C404401
:10550000484C4669726D776172652025735F56322B
:10551000320D0A00252D3130732025732573000DBF
:105520000A5479706520273C636F6D6D616E643E2F
:10553000203F2720666F7220706172616D730D0AC3
:1055400000557074696D65202575730D0A0025730B
:105550000D0A0D0A00564F5941474552203E3E2044
:105560000025630048656C70004E6F2070617261A9
:105570006D73004B6579207072657373003C6B65C9
:1055800079313E203C6B6579323E202E2E2E004430
:10559000756D70206D656D6F7279004C6F61642060
:1055A0006D656D6F727900637400436F6E736F6C1D
:1055B000652074696D656F7574003C6D696E7574F6
:1055C00065733E004765742074696D6500747300EF
:1055D0005365742074696D65003C595959594D4D96
:1055E00044443E203C48484D4D53533E00746400B3
:1055F0005570646174652074696D65003C6F666602
:105600007365745F696E5F6D696E757465733E0076
:10561000546F67676C6520646973706C6179206F83
:10562000757470757420746F20636F6E736F6C6522
:105630000062005265616420626174746572792051
:10564000766F6C74616765000080015000800250C5
:1056500000800350FC3F0150FC3F0250FC3F0350D0
:105660002578000D0A413A2000202025633A2000C9
:105670000D0A4D3A20002020473A20253032780D7F
:105680000A006661696C0025692D253032692D2577
:1056900030326920253032693A253032693A253076
:1056A000326920257300253032783A253032783A35
:1056B000253032692E253032690025303278203A83
:1056C000202569202569203A2025303278004E4F68
:1056D0002052544300253032783A253032783A252A
:1056E00030327800253034782D253032782D253031
:1056F000327820202573004D4F4E005455450057F9
:105700004544005448550046524900534154005303
:10571000554E00ACFA7F617C3B7749C65961FCA4C9
:10572000C825459CF46A32EDE1552C71706EE1EBB1
:10573000553584961D543CFCE250275C6A68244F22
:105740007650F45B0109FD4E82D9FD9D098719B29F
:10575000D1D2821B209DDCFF025834688D2A78B993
:1057600011A1547420E5701CB2689E22D5ADF19948
:10577000A848FD5F61E9BA322867B933A8521D8A8B
:105780002E7C1AE734E68F02147392210224638080
:105790003C1057C93B81A453CC834B30E3D9B54E61
:1057A000CB994F66A4DF92C0377C10787D02D05031
:1057B000E88DAD55AAEF4B1748DD329C2E609960FD
:1057C00029C56F2FF7A16BB4985727777E40E99CC6
:1057D0003809297E2616C4A4CDB032DDEC049B8A9C
:1057E000AC69CE6D5B587537C847ABC306D05F490F
:1057F0000DF7D3728C03EE6C76DFD40085ED66C7AF
:10580000C2B23F4FCB0B5D4289E5A8B21C806EDF70
:105810001558B5F4DE30560791D8A7337CD765D636
:1058200038BC521223E98259C5C5E5662E4B518911
:10583000A597E6DB6DBCCA66953D05F14033F5647E
:10584000FF55204B0F3868B15398DC78E76126DCB0
:1058500074B3C98658632556EA3B62C7A48FFB7CA4
:1058600073C83776A23A827151C2274FE67FBBCA0E
:105870008BD720AD5ADBE778D301872DDA6CC57B57
:10588000A8873C5B168DD73C99BB9F8CF5A4BFCBFA
:10589000A22DCF3E36C6CB3CB66CC841A93AFC1F00
:1058A000C68E20D283DE0E67DC71F34A36A26D24E9
:1058B000E1558C90C676296B70E9ED21DF64630FAA
:1058C000C8E42D7038876CFC4159595B084DCBD822
:1058D0005EE3F04527E204E16D1CBEF4C273E99F6C
:1058E000818CF866229A6D6C0D4BC766B2D6BB7977
:1058F00031B475A428F9383860CF111893FEEEFB47
:10590000C72E9EC1377A63C3FF931929310A12E06B
:105910009E98404CF69797F29383A62FCED2DF76CF
:10592000EBA9F9E65B7DD4F2009011712D81366808
:10593000593286A5FBF4687C95D1E5D14AAB60531A
:10594000D72FB09BC68DAC47E96EA6C61DBAFCBC6E
:105950008E6045B0AFC5E7D821BF5590F07798D697
:10596000D734D300B99C7A8C51905C11666BC60D0C
:105970006B2CAC8917F1058419F07BCC1F0E039AB0
:1059800087DC289746F848F0FB22F690AB219DB3C0
:105990001E7EF550CA1BF03ED59E30FFE1AF96CB80
:1059A000027E43652248F9A8F94AF9513B810080FB
:1059B0004C09365ACA4820B8C0DC4D72A4F7ACA5D1
:1059C0004A4DED02DE7E4E9E8727BDC8F7A2658A4E
:1059D0004F89D371745D53F288D8FC34FF9F3288AD
:1059E000F834CEC3291993FBA06F001FD9D5E91C49
:1059F000359509F52B311BF5881554BD0B44327BC9
:105A0000B65A9392B30828D23E9D1A9A37D6960971
:105A10002464448095841671B26D370247A16E6884
:105A2000119D8BE2CB24A77967DB0338E0D8287D72
:105A3000E1CFC200D6CBCE84DCCEACB6379BFFA480
:105A400059D0F21F973C9D230293FA87E311C25964
:105A50004BFD55F776B590C9B2C7BBAB784B9CCA26
:105A60004BE8592F21DCD3C937EC5F595C5F17181D
:105A7000F313073590C22BBC3C9A6D3CFF797CA296
:105A8000632A2D9AABA7A68FA670C3CF1AA90E7C46
:105A9000ADCF29C4A9477C829975142C063E88A9EC
:105AA0003DF8F0BD47D88FCF48814A793F42D30BAC
:105AB0003E4CD3376D49F1DCD5990979B367310193
:105AC0006A1186EAFC8C1C1729B0ACBC7E823516A4
:105AD000707A52EB4176EFD5B32C1D0350A871FCC0
:105AE00093FE9E70A6B43988AABE1A58958B83CCB3
:105AF00025DCFA7B1EF2AD35732724F9742A5EBBD0
:105B00008E5042326A3E77B3E8E78DE7EB349CDD96
:105B1000CCD84888FE7700499EB1D19CF25EF5C38F
:105B20000D1C5E6B2D89E1EB43319AE997141B4FF5
:105B30008D1BD133B8DEFEE25A0C91A733C6BD44AB
:105B4000954182C69CB75EB1EEC04BCEC37F6CA9B7
:105B5000334A5BFC93A9D0509DEB8E88053577D6F0
:105B6000F34BF59755C4D79F20038EE4245D77F45B
:105B70001909E472C3CF09B17EA13D13D8986A0315
:105B800075456FEFE1A90738B852B4A196006A8E47
:105B90008BE47803D5E2DC39170B3E9084B824B24D
:105BA000A9F11D3957B40887F11B7E0992EB8810C3
:105BB00053F731E2E084C8B8439FE8B1EA519D7DD4
:105BC0003C5B412C1D7351A891CEFBFE2D16E7C006
:105BD000BF72CDCED86026D77F8CBC85362B38A43B
:105BE000A144F34A12BE8EDD65B38EF3CC2098BF7C
:105BF0006E9695E7456BD35006F622404F825927A3
:105C0000EAF0616D8E501D14854F93E39F795132F8
:105C1000E363398D4B8F619AFB384EF7B555A199E7
:105C2000EBCA969684D4230FEC72BEC695E25DEE65
:105C300042F1BAC5711A857FADAD339100E354527C
:105C400074507D4BD129ECD47DA0E01F208FAD187E
:105C50003F7C721B165D806278050A836CA8753ED6
:105C60009A2A045A80245F18BFDC050149892CDF79
:105C7000022ADBCAC16B9706164EC7C61E1E958E3A
:105C8000EC8987092D343A0056B5C6558F2B6436FA
:105C9000EA01711BBA816A5003987DAEF1E1D764C5
:105CA000FB597DB706E0055B4EB08410A93FFE00AE
:105CB0005D2203FC86FD3E2E7BD0F353E7A8E92B43
:105CC00017F69917F9B0533F4A9D0B45C3D397F286
:105CD000AE73DDF18E0776C08F8F4C4BCA9802975A
:105CE000585306D7D1796143ED608846A465EA0C24
:105CF000C17363E7F5D9309643930E3D180A5D27CB
:105D000062BCD841AFD27408C0AA9571FB5A5AA49C
:105D100067AEFA5E0004E6C9D12EE3A8EAA1C31873
:105D2000A4B20F694A080E1294590DF5EB49A2ABC3
:105D3000579FECA01697009A876ECC27821872A402
:105D4000B3D045540A3B53EF6BB6EAE8083E6E9C6D
:105D50003CF6B39C88657FC0B07B4087B68D4D20F4
:105D60000E15607FDC8138D2E58A85AFC1A8EF2DA2
:105D70000BAC92344346E971852690B2FF8532A37D
:105D8000F753733C8BA2C11A548F752A92B382F4D5
:105D9000A9BB8A6201414C18EE65D5993ADFFAC673
:105DA0000DAC78C3EE87DB9CDAA767CD7E83C88B0A
:105DB000D7663C00C54FE9B4DB92BF591983C62BA7
:105DC0006B458C8E5FFCA2598B936EC240D5C5E9A2
:105DD000A1CB8CE1783F6AB57AE783EBAAD29185B3
:105DE0008A744DA232B1766CA21BEE3C0A44652146
:105DF000B59D8164BADF3E0A5481260BD2696CCF0F
:105E00006A90577D3519B3C0B122B175CC5F080CCB
:105E1000032A805E01A177F3B0990926324A955B87
:105E20009A8512483CA8B2DBF1CB498228725EDB2E
:105E3000686B7265FB88EF3F4FD039A1231142DEBA
:105E40002D61334EED84A5B694D07C96186B4674C4
:105E5000BA8BAD36AB2A98A2FB6F42B1F42D034A40
:105E6000ECB887478007F545D9A8A8C1393E9833D3
:105E700071CE356E8D4F1FA37A0E5A178547255D5B
:105E800076F7308F75A1D4E749663E2FF20662F7A8
:105E90003B18CB836F863F31682F95CF7C655EFAC8
:105EA0006BED5FF67D408E4F6459E044EABF04D449
:105EB000A4F5AF9EBD3EADEC24E98B4263AB6F3FD2
:105EC000EFBECF2771AFBA111982560F9C9A764850
:105ED0004DABA6B87B07B4BD6A9FDB73C5D4F9B3DD
:105EE000FF3DACCF226AE4DEB56CF89BE03251DBBB
:105EF000BEBEED80A3123110FE49A273E61BE4A5DD
:105F0000794D522908357E8A2C5AE5165C5A2F2085
:105F1000120BF0CABEA30918EA90CB9CFD666F9CD9
:105F2000D78E8ED60199A248012FAA669445391EB4
:105F3000C326C6F0FE240DEFDA60108B9FB70B98D6
:105F40009A9DA84FE131F45E1BBA37B4E13AB2062C
:105F5000EB105DFE922980DF7E330F13E3640C4E5D
:105F60005268DECEACBB95729C763A14F09B39BD7C
:105F7000A50A71C7E65E3F2A6D38BB9A983DF83E88
:105F80003DA29A1301AEDE225FC2AA21135EA5864E
:105F9000BB2AA8D7274859AB569C15ACC9CF8B3D17
:105FA0009FAD14680139C3938B35FEAA9D05622B02
:105FB0002AD11D40A61AEE77F06BF69B15393EE705
:105FC000F759965B7533B4DFAAFD872DA7E8FE511C
:105FD000605E0F6AF9FBD64C11FB4709B4E67A54B0
:105FE000F5574D7A5930F79088957A7ED33D3A32FD
:105FF0005C7BC98BF3EEF4BBBB0B029A1FA6DEC21F
:106000008F558F8632AE6584E3EFAE626EFDD6515A
:10601000E0AD0F8DA4075349D14238A0CCD322E77D
:10602000C41621508976133010BCFA861B2990FBC8
:10603000F0EB4784A67DE0F682653D59F582A02508
:10604000A19F7E72850012550D4A017D885CF8295A
:10605000DC7ED17639E1EB5FCC59E5F29BD61E169A
:1060600084C9B5F89DE8A6B757447F49DFAD7D4D9B
:10607000FE14A7DAB6A71B24A1854ADDF9B1063BB9
:106080009DE6757C92A6ACD837FBBE6A880E33714C
:10609000F2DADCF6D336D139830417717FA78D3657
:1060A0003616152BC28B8D9E3B918EA194651128BF
:1060B0001C662FE6BC6D71F8066712F74A4D33086F
:1060C000AB4D111B54D747AA7E1A9941F81C945C1A
:1060D000C905448D1B259F5B0B79F023582BD1A656
:1060E000E983BB0A33E4E5088DDDD2AE63752D3D4F
:1060F000858BBAEF8E03CB1453DEA0E9EF83410901
:10610000BBA2432156E00AD00EE94D748E454345AB
:10611000913410EC348619B58563FFB8755CD6757B
:1061200077CDE33440691D9E58BE3E109EF15CB6AB
:106130003D377F4B3C6A92C43E21034E20ABB5AF46
:1061400051DF0E51C7A2AB14EEDB25A575F1B69554
:10615000245599603BE10E15E407C5F425C465009C
:10616000DB5D8FD8D09FC17629A3B2ED5B27D29E8D
:10617000D99A0BCF28DD01420F7073F1C085DE3C48
:10618000F665086F2985910C1106351C81A5481309
:10619000F4270CD2902D1498584489703449B7C113
:1061A0000138337046D4CECE38DFEFED1E4DFAD72E
:1061B000651E7B6A832078C998287B0108FB0260F2
:1061C000A652682633298F08494D6D1C19032FB438
:1061D000607413BD134679AB9CFF8F8D1B6D4EFF12
:1061E0006FFC4BDEB089D848E12CB91261A1683947
:1061F00082359F13201E93D05DAB11D69AFDAC0B58
:1062000069F4AC1E5D7E0D82E59D77DEEF1780FDA3
:106210005246E8DEDB9826FD30768488FE257CE059
:1062200081A27E2E90D65E31771F10BFCC45F577C8
:10623000110CEF9166AB9481FFD511F146C7104167
:1062400062144E24C7C8C9C033AE63BE0BD7D9276A
:10625000214C013324F3B52F0A9DD99DCCFF45CFA6
:106260000965BEF325C718F2AD113C620BB76C2D62
:1062700018E76003BF35BEBD3C17B8EE4C125BC3D8
:10628000E476E948862CD3D8A0E85308F03AE7E949
:1062900066610DF374FFCAE2EB8BA69CE6D4BDC821
:1062A0009BB185B5D93308B78EEACBE2AAFCC32FE0
:1062B00060EAF18D2F1EA6206F7D4366B1845C627B
:1062C0001673D39F3FE20180839F6EDA8B37E0D352
:1062D00068AC266422B0606064BA0AE18F003010B6
:1062E000E32F57038D7E9B79A3055C1AE8B600C5A2
:1062F000EF06E0A073847B29F980628567F51BAD0A
:1063000064BF769D6F06EF950F5B91106D165FDA97
:1063100092B505E5DC5336BC84F48019D4906DB990
:10632000FFC0FFE301BB8187F8541F168F6ED9B5FC
:10633000472F3389C1723055CEC1C08CB43C1C0B81
:10634000506923A3D1DD4927CAC769F2BB851C5612
:1063500007FBBE9DFD61F38B0ECF9C68A8EB6085AB
:106360000B65E77124E0B66BDDD86B7849D81F6206
:1063700096E840ED6027D008EC2ACA0518DF645380
:10638000FA08A1BA04760DC4CBA30FB380C39CBD99
:10639000C89AA6F47F3059FB1B00E95E89B6B41C8D
:1063A000270BC9C420367D622EAF2F8B5F96C72086
:1063B00007863EFDD00B91CD02D624D2840520FE67
:1063C000DE6C355A0DAF6BC9CC2332BF95099E7771
:1063D000E799A515FE56041D81FFEDE66E3171F4B7
:1063E000757CF0AEDA47E334556D602CF6AD9EE077
:1063F000A50E413FC4266AE332F7D8D7AE1431D593
:1064000059ACC590D7A52E61CBBCCF3E5D719E9592
:1064100009E3B410D26C8DDFDB37C71FD243C87ECF
:10642000206049E01336C7B08B505C8EA934248BB2
:10643000A19BCF0FAFF055E22C97C731BA7F45A093
:106440007F8B3E5EDE6A747758610B6F7E02EA5086
:10645000D977069EDE73FA039DB89A650DEF616DDC
:1064600059F97EADC4334ECA6CF2D27501D58FF5A1
:10647000830A63A28BC15B17987BF01E7BF0370801
:10648000E8FF3901490CAFFA22049B1AA88CE333C8
:106490004750274774B44CADFCE10695B2F5A48C87
:1064A000D067FE6725739E2CC37A86BBD15997812E
:1064B00043A9C9674AE467091ECEE9B8D417EE2B91
:1064C00036A98038A5A469B5D6D2E39E7A09943F4F
:1064D000C356D7FF64E8FA87220D653F0DA6042452
:1064E0002D454B1A581DA40441DE94A6511F158555
:1064F0006263107ACA96E7D8F39F579FB782457FA9
:10650000C15B1733D4111381A0526CAC8201159A70
:106510007B761BE5D0341AB827A9A32BC479F709D9
:10652000B57E05DF57F30ABE3591513D0EE6EEF715
:106530004767F0A5E5214D216A99425E99BFAC7588
:10654000EE70618918763D32E173D6F74BEE4EAAB4
:10655000BF3A5E3900887B645DFDA03237C3FA081C
:106560007569447127E697F441D6FC519616E834D4
:106570009C4532F11E4D79E3AD27FFAD671DF43A1E
:10658000479EC70004AB98A5E485A33C477EA4536F
:1065900059BC5BB5A9F72E810B101B4869C5051BBB
:1065A000AC690890E9F8C0FBA81AF76B623CB50823
:1065B000E11379B06A53B03C235123E65CD42C50EC
:1065C00011532A03E53D877E188ECDC1164448D06D
:1065D00068F1DD6505B9530C55236748B0021B0F00
:1065E00025646A501E4D6B1C25BC3D7193FEA11F96
:1065F0001A416B5644B28250B39DD762C5B2BCDA21
:106600004AA8CD49031BA05F00F3F3EE93C4B9B7CA
:10661000EA8071C02BDDDE94FE34838662237175BF
:1066200012782421409F9D2FB4B82FEE6F78D5BAF1
:106630002E2E38756B7ADB9FCF33A6032D3BC5D04A
:106640002DD048931D4BE30DB6756E8984723427A7
:1066500069D7C1F4B8CC9C830B541F87B13A85B776
:10666000391AA979052B7A51F2F845835016EC694D
:1066700091B446413D28EDF2D95354EAA5AF24CB5D
:106680006291A6D0838997A1BD1A6BA52890BC867C
:10669000596BAA1EE72B42DDB32F28B5A6CE5DFFAE
:1066A000E0A7BB500D5E6C1D281E5D65F1093485A9
:1066B000F6514CFF8F2A1C68F4FD6B5085E33E08B1
:1066C00043B07DC22502102D73C3BE4DB57CDF7172
:1066D00067AA6448FC0D95C7A0940F27EF5A59B6D6
:1066E0002EB070D1C9D2E9E9AA7BE6984E4313EEE9
:1066F0003FDF82D8AF814F49F2A9CA9267B6AB6536
:1067000099A9714AF14FEA5201B476D87C273287B1
:106710008F03B15DE9616FDA89BA795BDE8770F169
:106720004984BF33A39B31E0006794E0B9910C2307
:106730007AB9CF737ED7E052F6F58030DBA7C86414
:10674000AC4627EB3DBDB5BE1D574E1A2D82F091CC
:10675000DDEDB569CF51FB13222950AF74077CAC36
:10676000261871F3969B69F74CCF69A10D48B58B3C
:106770000831FD2C2AE65896D88E816DE61CAA7544
:10678000EED5E31C04B4168C3DEE2C17795A1EB0DE
:10679000300DA5355FC844C1C843E660F666CF1228
:1067A00024548A63F16B85645C124F43AD842DE2FF
:1067B0001A1F3D6F195DB2E9E5AEF4E92A5061395F
:1067C000D2D44C90060E91CA9B0FA3B64AD0DCFBE4
:1067D000707D2938E6388A083BC1120B12B4C7AA6B
:1067E000B5FC7EE056F6BFBB7EA6AA7B653CC9F72A
:1067F000695EBEF9FA194463D029EFAAEC41AB7E79
:10680000D9F1F988BFF875851839430B639D639FEB
:10681000C53040C22A5927096E33821C0C72B73D1D
:106820004CE214FFA8C9D1B7D4DCEC46E6E12EB1A6
:10683000E451365096332C4A02DCF0E4B1BEA93B59
:106840007A27D467C4F6E124678C4BC867E3D7790D
:1068500020597482C8B70D4E5866C23D6DDEB1F442
:10686000AC0680234B1FDEA8A066B97D87184D8A31
:10687000F500B2BBE8577D9E52E16934453F4C0FAD
:10688000158E6C94A0742E73A95244620C709751AB
:10689000D16EBD8F7FB02CB615EED526FA690345B3
:1068A000A0F9696F50F5C6BD05DDF548DC0820CCC0
:1068B000875AF7C0328D36A3DEFA8433B93AFF180F
:1068C00073713ACA1C5E83D6E9BF1174AB375FBEE1
:1068D00086B9B1ADDA61E4BEE2573B8173FDFA815E
:1068E000436951B7DFB4673BA55FFF5191044C7E0C
:1068F000BE6F4B01230A701DF3DDC14610DBA7C23A
:106900000D68031720373A64BB1AB89254F72D74F8
:10691000C1373B8D4A7A7E9AADA0DCF4F953DC8016
:10692000857CB9B508317A92FF5552265CEF8758BD
:10693000312391F5C6486D8C6721105838130B2B05
:10694000187CC415DCC5837841B6A4BA26BE871A64
:10695000D986E0D43D3E98684FECCB5B12812A5B30
:10696000BCBDD1F866819ADE6288D8BCBFB2B2F8ED
:1069700094501DA9EE4ADDF7281A9EB728ECBE0AEE
:106980008EB7DA226123DCA5A38724E1794438B4E9
:106990008C6827573844DD145382AB2CB1DB16A327
:1069A00072A993FAB95C0323FB8B78411B639BD7D5
:1069B0004FF608F48A3C6F45623ABE8D9A6D12BE5E
:1069C00017C654B59DB94331FCC364EF934B9F5C2C
:1069D000ED373DD37C110945AC55DEDA8ABDA28086
:1069E0007713D1A3C32051832F20A2E11463D6359E
:1069F0001E98F9D929AC0313A874C13E6F27B5734B
:106A0000C59E4DB1CCA55A117C19C9CC6BD2F37976
:106A10000BF125A3BAA3EE6DDE6F92E33DBE9D732D
:106A2000E938E06ABC188C9D8758269AC1252B212D
:106A30004D9A72D14ABF0C1877E358ECFA6FFDB744
:106A40001D32A34F41482E13086DBCECDA58E17794
:106A5000639F83C2358E8B665906B7E4DDA3C44CB1
:106A6000F5589733389739614D6CBCAC50D9C09903
:106A70005B89D93F058F6988E5BFE07FF55189269D
:106A8000583FCAB169FB5962B729BA5D528895F27D
:106A9000BB59898F46F6A5A66FD14FDAEC373782FE
:106AA0007F756384AC8C0A4F123DAAC415B1D3091B
:106AB000B30742D8CEFF99C3B4B69A0131263CA998
:106AC0005E0F09B3683F8E5E8D1CC7189DED33269F
:106AD00076B1A3700F8ED8C35ABC32B4D7D1F95651
:106AE000066FEB1BFF1ABCB43764C5984C830D5C72
:106AF0004BCD6C43C99C7BBB9C3CA7A5FA4F0CDEDD
:106B0000570F9C364A225F984A90F6DBE2DFFF235C
:106B10008917873DC73FFA358759ED9D04A7B00F08
:106B2000B3B9495B692DF031D1C80E36BFB606DC6A
:106B30003D1B65DA4164202BD17ED47101CDB107B4
:106B4000CB9E03EEBD453F76EB06496012A88D6AE9
:106B50004BA8650220EDB409CAD50FEC094384B7F0
:106B6000043E7CFB40B9E41DA81DD9AAE1C79310DF
:106B7000C4DF99B1DF374086ACB8AA1D3A7501660B
:106B8000756D1C34C1914A62D2864C3EFB6FA8E8F9
:106B9000EBD61BB9C5FAB5B157CE65E58433C8A4A9
:106BA00011FBB6E92A79D0AE7FE70E6EAB1A6A63A5
:106BB000F3D998EC27BC13EC0BDE1CB5D506B1B1AC
:106BC0001BC4A004DCB2C5DD98A1115BDB6217D940
:106BD000B5E00E5A4800AFD08CB6423B0282FCC8EA
:106BE000378F2D85A7B03BCDDBC94CFFFE159DDA55
:106BF000E25ADEEB08A921FA517FDD71890E895F27
:106C0000BFED13D54EF80AC0C97F5E3A522DB38648
:106C100048907F04E2A694779F94142F5621AAF3FC
:106C2000B9DC689D2C8DAFFD7C6AEDDD9B879F7183
:106C30007172FA109CC0B26D05B5D7719D06A41390
:106C4000557F4BAE2CDC077658270C3EAFF366AB76
:106C5000E28ECBBDE229FF5BD350255AFEB1A3D80B
:106C6000567E285262992130C5906E0A807AB139D9
:106C7000B1B6A5B5CE2E1BC8A8E1C17083B2D0AE07
:106C8000D3A7510AA834E06610B001A5E7D1B53A00
:106C9000204BFBB41E236B3FC00D6958996B0186D6
:106CA000B2EE0BC7E537C6087C3F985977E5E7D6C3
:106CB00067A09C98A7586C2EEF9960049D78A2C19C
:106CC00057EEAE57F7B2868DFC013FBF2084B2A4C9
:106CD000E3CC8ACF607F6ED79E999E4E106073E79B
:106CE00099DD4B114130A838EAA0872C34718238E5
:106CF000CE046BDB26DEDC161FF28B51693EDA44D4
:106D00004670C15B8B2832589283A79B46F989A0B5
:106D1000D9DB5A9CD32A3BB659205775C241ECD5D2
:106D2000FC69E9F6EF98EE9B501DBB8E290357ECEA
:106D3000BE0151084E2B51376C676124C039F935BB
:106D40008FDAC80C85DEE9C70DD814C38B7C1229F5
:106D50009E23D6286A0EA73B09FA88825F257C48C5
:106D60006B139B80E788870CD08FF921D305AC2467
:106D7000B04451310FF55F5AB61DCE1240354D2B40
:106D8000531B5A5E113A184CF26D29269E1CC305FE
:106D9000A52084BB7BDE659B5EA00237DB621FF70C
:106DA000AA22E7203FAC2301D0CC5ADA002F96B8B4
:106DB00089F616EABA6824B7BE058ECA11D41D2713
:106DC0003EF3630A9F176D00DC5FD7908B342F98DA
:106DD00045C93A90F7CFF35A6A084FCDA7CC005077
:106DE000BC06496263D372CB76E426D308F5A306CA
:106DF000944A8C1BAE5F6CB9C962CCDF2348B9FAE8
:106E00001938D6E3876406C3E158917A6536EA8873
:106E1000FE7990359C2A697294EB06405301711BF0
:106E2000B012763809D64B042BEF156C8A79B9FC71
:106E30006F5E1EE364451D8F7119D5D6D88818B3CF
:106E400011A113B69998A8363EFB6D97DBA086E694
:106E5000197282D4868773F3A0B5DDCCC9389EE65B
:106E60000FDCEF901CFBEF0179DF6FEB91F59C36A7
:106E7000E8B9673E474EDF143B032B0F92B8681EFC
:106E800001BBC28EAA98D0E7D6519A1C91FC15413D
:106E90008414BEBCD852B881D5B890A292FC036FBE
:106EA0003444519B0FC50AE41C9E532AFB01BAC00F
:106EB000BD00FD9CDAC0B3E5FB9C7373DD44E8F4D0
:106EC000CB7F7066C6D6E6ECD30A4C26DF212DBBFD
:106ED000F2DE689E8EBCCC0F0F0A774433D592E168
:106EE000595B07EA07372936FBF83C0C07EBE7B09C
:106EF000AC5B5888EEC9B10D6BEED8DB8C2B8E5E87
:106F000079349CCD477D120075AFFFAAF1230E980E
:106F1000ABF22C804D9401446140AA763C853887C1
:106F2000149C5B1C7E195BB705FCF38F656E007DBE
:106F300096C3D856DD164353C5E3143E026C36861D
:106F400022DDD13BDEE7AFF9C77F0E2A395B5F1840
:106F5000BF10B8CF114731A11A216D82A2ADFF7EBB
:106F60002E32A178A78252939A2E7A9A60555A208F
:106F70005366C51172FE1ED72D353782A5D2C03E8D
:106F8000B074A6307909B1D24267311E0F706CEF30
:106F90004B5A155C477C6F825389A3FFCD7FDECEB1
:106FA00063018A1131C3E580EB9E77C71285CEDA83
:106FB0005E9B5C7157565E07DEBDA7DA9B959B5EB4
:106FC0007C08936FD6C32EA3EBE1DBC66E246B97D0
:106FD0002CCE3570D71D5195A6B5BD6CE3306C59DC
:106FE000BE36D1EA62CA67900762698DA5A925E518
:106FF000C200B4C257B612762A577DB4D2C5913CAE
:10700000B863FB13E6353DABE0A796FE4F2F30216A
:107010005EA40BB85B6DABAC40097345C3A007FE23
:10702000C6FC9BDC45F83AF47786FF13D71B3B6719
:1070300084C7FDA1839459F99764E6B078CD1C57B5
:10704000A17511846DC055867F7D3552F04088B2A0
:107050006B660F3505E36167381C9354041AD247F9
:107060001CD937C51D4CD0620D9C50DA6F50FAA662
:1070700023C93DEFD99D86A32EE64E0DAF34ACF962
:107080002CEC278BE733A39DA9F1400F7F1AB0D0DA
:10709000F5B0289F60B811447B5742A39CBA515E5B
:1070A000AE2EC4D35FAB5BED4908DC6C815D03F2AF
:1070B000E8AF8D1AF2C8500FC7A7971A2756EDFCF4
:1070C000C5B67AC790CE00682D5B9F022714C34FC8
:1070D000EE7E2433D080436A21B608B0B4C3DA19F7
:1070E000C2CF0AC1AF4D34847D2FA8819D7E075D3C
:1070F000505BE768CCCEB4AC23474D07E83A57F174
:107100001BAD4A55584B9067A9CAA74EC23ACF50FB
:1071100031A2A3891A8B48957B6E85F3CED5402189
:10712000202DA4E0A5D3DA885957AFBBF48D7CB6E7
:10713000586D4CBE3C12F0C1FC535797BA342A43E9
:107140008042A24FD538940BBAC80C7880D6ED7C1B
:10715000D171F5CCFD996F5E3FA85041CED4E1923C
:107160003840BA5E7CF247DAECF039D8868946EBD3
:107170004F097571D90029813A6CF24E2A9EC1AB34
:10718000517C3F62655D7E8F5071E0F70C5AEA9347
:10719000AA988610D0E4C957C49CECD6703A023441
:1071A0005583D4A250DD6E4841D0442B55A16A16B8
:1071B00094BB54B0709036FA824BF77A1ADBFB26F8
:1071C00094F19A5767D1A3631D6564E0EE909FC95F
:1071D00055610CADA8DECA3BB3E8E826E689CAD003
:1071E0008D89391856EB283F13976ACCD24680F226
:1071F000F4D1068AA77FC52A4AABDB24E467A188BD
:107200008C9C3CD6C7E6C13B6DE515A9422E8E315C
:10721000CF2661018EAB420C1D9057234FBF3856CD
:10722000B0C13DAE53FF2B76F245FC566C4C724616
:107230002D7A2EB310F9A2F88A4C8416C15025205D
:107240005DD6B69368408998D9CE59724F4074295B
:107250005FBCCA7A425CDE877C0A413D9E123F8851
:10726000020F820D36B68C9E71D566F39BBE43D954
:107270008FE4BBD602F9B557CC449C6A640E54E344
:10728000BCEF43E7BC86463B161C6573C1EC88BD6A
:1072900069DBC8DE8522468AB7926186E1641F50A9
:1072A000B5B959E41AC401B5AB2BAAA5FCADEC8461
:1072B000D289A6013EB8F2E1977745E4ECADEC96B1
:1072C000065782958B968ADBF3F4C2D1D206699574
:1072D00041FE94C49441D24548F44F5302967FBF77
:1072E000CE2B3C856377A4C8E1886D56CC986C485A
:1072F000EEC3B0DD740F01E0D133C2B18F7E35B380
:1073000053E6A6715933DFA4F96FB08705BF6EF05D
:1073100026B530D1F27ED4CC77C9A815CE274366E6
:1073200096111E577A97C29A212F9EC51280B07B64
:10733000E82ECAB439B55E6B3F04DE21D9B5D92435
:107340005F0E347A0C00DDFCD581C7B5D8B6F68364
:107350005B7402659B010BFC6BD38FAAF81787EA5D
:10736000F54370C723E68CEFD0B0009FC67C97F83A
:1073700037B80D725E0359F916F3091D4D455DC10D
:1073800036888071813125525269510972822024D8
:10739000C547688243EBBF8AAC80D39E7996DF34C1
:1073A000E14FB391FDBD7C37C5860660C2979ED282
:1073B0002BDA1203C99E360F4EFB97BC56A34B86A1
:1073C000EA856F2B5310631C04D17426371F8D1769
:1073D000A3DBB5A50742962A2CA8D7C1D63D7F08C6
:1073E0002B37700B96D780E6DCBB56D2408B799555
:1073F000F638CAFE34DE15004EE426E9ABD97FE745
:107400005C48008AAFECCC264DE98DE17C746CE9D8
:107410003371BF7C8E44F1902A6715C8D61E57750C
:107420005565AB44B6A3D19E329FDD930FDC81C07E
:1074300068A49DF1AF715618A68046404DDD7B8B48
:10744000482C82588B7D683588F9F50944D9712715
:10745000EDDEF1AA11DF66B93A75AB01FA773D644A
:107460002917089DF7DBC062F791B66E84825488B5
:1074700044427627B9B7F3A96EDC2FCD23C1FB8434
:107480001091F0C132106276A037C4030D791E0945
:1074900067B12B6680B07EA611D22BF8F0C38A8E1E
:1074A000768B084644426CA7A691FA3F38D35B6EB0
:1074B0006AF810BE6F4636A8AC47D273964D0B8261
:1074C000722CFBD83D5F918D5CB09BB5EDAA2C630F
:1074D000C296EF8B925656ED289C97F4D447260D12
:1074E0001BC6742AF3E0054550F35C7EE66BEB7730
:1074F00082060FFD65CA9C922608CF497A775D9770
:107500001175AC3409285278987B1469B86578C62F
:107510003190CA4370E64D3F3FC28A75C7DC1AF509
:107520005E382280444951DB76BA4B3024141B7AF2
:1075300078000F7CF97F1EB9942ADEDC7DBA77BB18
:107540001A0165E3BD471B2F4D1791D5DBACDEF863
:10755000F8A1D83B3200041D1766C65DC030812EED
:10756000481C4559CA0812CF93A1D7D5EE41329293
:107570007B158DDE9FB31EA39A9525C39746853450
:10758000799E11C314D4EC476672712D38444D6B4B
:107590004F27E915EDDF03D7DF4A97BE9CBDD19C8D
:1075A000954DBC89DA527C5D27D7646879479D91F7
:1075B000039AE0F0BFE38CD63243C0ACFFEAE5E3C8
:1075C000923FA80097F02C22D70F13E49C0BA8B889
:1075D000C6FC0734D0E1769B296EB02E8A186FACBA
:1075E000EC8267309BD49BFE2E4051952C426878EC
:1075F000F69E1C38EC487C31BC5591F264005690E4
:107600000A75FF29BE90C3FE7BD0BB7DA41C441825
:107610005CE7060E9A62EC507B6F087C3FC9FA7BF0
:107620000EF5A4BB6563C1DBD1BFE2D0C581B1CD8E
:10763000F23D9F9FAA710F77E6DC50635A243D26E6
:1076400096DF2618C8BCBC338F2A5EE10408AA9ACC
:1076500000C0BC1A01378D1972627B1AAEAE3B3F77
:10766000960C1FE425CBB8C2E2B87DBC179B0497EB
:10767000904A81B3B53D4885E64D7EA7F994B36144
:1076800093E31BC084F09C3C52B76DB65F99345CA9
:10769000E55F124BD450FD748195907AC7E5976AE7
:1076A000C45C19F9E2AEC1FAFB977774904D76602D
:1076B000E5EF9763C1C2805F5B0A812477B2D5E9A9
:1076C00054DB293FBCC92ADACDBF140B75B280C484
:1076D0003D6EBC419665CECF47D2F8FF9B575AA06E
:1076E00066B5A25B0D11834A05852C9183E646950C
:1076F000A7D0C7478EB8C8D4491B5DD92D4E36E6F2
:10770000A8EA52E8043884EE9AAD1AD49CBBF40A75
:10771000A06EEAFE6360E4367881A9ADA75E2B62B5
:10772000624E22D6763E6D7A25E86E79F00FD83912
:107730007F38D6945C220D2FBAA87002A709E7A95A
:10774000FF73BA2D7B5BAC817B6B810103C9A057B2
:10775000BFE0DA486F831B4FC49C941C3FAB753E5F
:1077600058CD5E97B3A8459C0360BAEFD8698E2ABE
:10777000384CC2362826BF59376098CED048F868B2
:107780003DB6B08543C2256F9044243A7E80D16EC9
:1077900045E1D4A8B65615E28C5AE4A719E331C0E6
:1077A00004E19070402854F561BCFCC875782C4EFB
:1077B0009CD468BA505D2D438BE9EA715CA59CAFFF
:1077C00060E787D8374F6FB75E6A5A4DA114189497
:1077D000E56155E18251888922D17D7B484A53F980
:1077E000A8446258486568AD97A0BAE47003EC639A
:1077F0006CE8D7CF0F0396956408A4F2007E61244D
:10780000AC174F03B08496A4284F4C423852EC88F2
:1078100085BB216F7ED1F36E7E380E58518F4C623E
:107820000DEE838100443113CEC981B3A1CEDF9B1D
:10783000259EC70A80004AC79E777DAAED9DD38307
:1078400093F048849558B3DAB52C42B3AEA5E2F074
:107850004A20FB8B15705411CDA6A7DF763B42DF83
:107860002255E7F01160C0467131BD825CD52747D3
:1078700044EA849A8AAA3C8ABF7235491B4194B46F
:1078800072A8DA1A90B24FE4B40006E680F8F4B3B6
:10789000B3057A3828F556F88CCD94DB88855119D4
:1078A00095B915D86FCEEC555706DFEA069A9F6951
:1078B000CB2F1DE0C3E59805EC726063D4D6ABF521
:1078C00068A95210459BA729B0F4E9435C5BD51722
:1078D000E0B3BED1BAE5742D669BC787BF4BEEE31C
:1078E0001E3AF5F864B81E07E3BB0B3E073B518513
:1078F00086BBAC5A33CBF54948428E1F39BD0A1CB2
:10790000778C99B6B604DA07CF214D0A5296EEF479
:1079100005A5CFD93F8975CAD13F3D5ABFD71D981C
:10792000914EDDF7F9F6D4A12ECE63F26A39F1D18A
:10793000ABE63D14D3AFBEE5A6F24E4F73138017EE
:1079400028A1CD672BD7FA7F6F7121E9D1F4186E8A
:10795000CCC198FDBBCCFCDAA0560AEA4519C90493
:10796000AC68B5889BA97148B85E02D05829A0FFC1
:107970000EEEAAA1F744C3827493A23756B0202515
:10798000B242018E1093D41C738BA1C35CE86DCA04
:10799000CEEB21C9C78C7F2AEF6814C98F22EF6B09
:1079A000BF45FED470F3EC52888FD60FD40B79E626
:1079B0001E6BA49ACBB5B9FC6B19A134C619AABD2C
:1079C000400A6C13D39BB66BD5E7D471797D5076A2
:1079D0005694678F151D1705D50885F724D6E3AD96
:1079E0004D57F9700D867B2509219009AAAAF6C585
:1079F000D69DC4E849E2B04DC04C55355DB480B564
:107A0000D5CD5E7C4DA84F290D6048DCD7D889B410
:107A1000B38600BF6B7322DA0C200BC91E9CB31C0B
:107A2000BFC68F11CEC7580DF0852BA045FE2ED3B3
:107A3000EAD17B67A070506EDAE78CEAC4DCB0DC78
:107A4000D35A6ED7A3439012CD28EDF3B78C8B1980
:107A5000118E90663A30D48AB69E54C7A89D4F1DA9
:107A6000AFAD6E131E0250BEA0E500007DFB758118
:107A70009DA14B5F3F561F08D6C806C36C88D6D25F
:107A800048E6EF699E50CFF6E2D630F9CC1C77EF8E
:107A9000E488230303ABD40A724E26ABAF9115B032
:107AA0001A006AAE5C229A81BD2D98495445D5B61C
:107AB000C7E8EE8A4E243215ED0E47A4450F359CDB
:107AC0001F278829C47D129222FCF644B93CCD823E
:107AD0006B368DC50E484919D4EB2E33D889C5E3D2
:107AE000FC314F964E6BA56F38DCAC350F0C2CE893
:107AF000AF671D4808DC96D2DDA828D869AE93AAE6
:107B0000E0FBF462DB4C16BE3B0873CD2E9D2B16BA
:107B1000A0EDB0F5A6B7597AAC5CEE4DA125B96AD7
:107B200036D028373CF9E51BCC5D90965417081ADF
:107B3000210A5932BBB54307087051CA966235987D
:107B4000EDBEB799C566243AD6FF4D886E3C78D90C
:107B500058239B98F5842E3300803CCEFB1C3F17A6
:107B6000579BD3F0A7EC2D4CF684409864D11DD8D8
:107B7000700CF4D534B5706C7452EFBF5B828DF22B
:107B8000F6923EC4875BF19352988B9138DDC443E3
:107B900059C315513CA9C34420A9336BB1DBF1543F
:107BA00099F70182F6466E20B548E33D9AF088E6E3
:107BB0000EB1A2BC0245DADCAA0A6369D32E559045
:107BC0004F0E84BBA8D48010044EE27D27475DB5DC
:107BD0009513F85FEDA4EEE7FCC40B5F9E4B1840D5
:107BE000425976FC90E2ADA456AE9239C177E38D4E
:107BF0002D3F7859B24F7C7E32F5308C91719232A4
:107C000011E3DF4AE886A56D8978ACF90BA33DBD89
:107C10009745E0999391E4130637D939F9F4B1897E
:107C2000FE250ACE406E82E496F1551C32C21D48F4
:107C300024DB4628C0BB3AD382CAB805B1FEDC05B6
:107C400041771F29A84DEC1283739D93F191A77D75
:107C50001F6D6774A089265925597843EA29249114
:107C6000529CF057E09BABB06EE2F60E04D51E605E
:107C7000F35F4C0126DFC80DABD2D4F844611DD3AD
:107C800063A9E4AF0B47B29FFC7683771F9E5286B1
:107C90005A0F9752E2DFF168B914EEF0D03412C4F3
:107CA000190A2232371AC5A6EC0A6E740C396E9C7A
:107CB000B758074FDC12B6AF5E8B95065A18A72748
:107CC00020C4BDCE9F375B4ADC6D7A1974B885B786
:107CD0006C66E3F76AFAD36EF365D80C8583F4B368
:107CE0009BF019D2890E87611EF200D1FD71AC1E86
:107CF000B90F40FD20FA29EA7D7B9F0928198C964F
:107D0000F4DB80D1DD657104B182FE6B262C446A00
:107D10003C68987A04F433C09221DCE2C232D08706
:107D20009ADD132E3DBCF3B4FF9831B527AA4B2141
:107D300023127BB411A3D7C7CA94D426B5E5B008E3
:107D40006ECAADA97A4CA9A11C550A9D1176E3D340
:107D5000B5F84E2043279CCCFA65F3D3980669C04A
:107D600026960E7D9DC0E7BD73D1664A3BFB6F2A08
:107D700090C5C488BF0791A57922E27C5555DF44A0
:107D8000C860B9995AA59B46B644B7252CBAB34CDE
:107D9000C585AD706A8A0957AE6E764C4B0B0E13D3
:107DA000A6276E881C10E41E69122023CE4CB9153C
:107DB000954DA8EFAF1795B341922C92E8F343BAD3
:107DC000F3EA707296848D84D81D6BFD1211157EB6
:107DD0009F501E5C9053F553546A064D6C2400F876
:107DE000E1ECF1C38D0049F7F41770C87AF35F2E08
:107DF00028403CD2CE6C561C07573CA4A2AE8CCF78
:107E00008D50F0E5DA5AF9B662EE72DCC23753CC27
:107E1000CB55BB26A115A0D94B3D53F35C5CF7E1D4
:107E200016CCCA9A35F4A1837DBB7CC7872DFE5939
:107E3000F685D5208FD54E071758BD645958D30EF7
:107E4000BF48D843F7F7D3F50FDA26B57EB197DCF4
:107E5000094611736FB7CD90AFE1A8128682A3993E
:107E600031AF74323B76894CCFAE888B96D5FA4AC7
:107E7000754CB61C4E2C28423FC842CDB529620B2A
:107E80000175266E67645B110E828559606CD5534F
:107E90008C2F7B911D4CAB258D2A95182109E5ADC2
:107EA0005B5823B54AD2E892156DFDB3727528155B
:107EB0006CD368A22BF9975912D612443058AD648E
:107EC000616354A4FE46677A31C860F4D34BD9D3BA
:107ED0002E14C52FB14B53FFA7A520DFC2D01F78AA
:107EE00074904BB73268E62E85F18DF81063CF7E23
:107EF0004776A05B69B421B857E8B3B4A0BFDFB13F
:107F000088D88F75AD99DE45D01967E0CA06A96497
:107F100063887DB53C064F2800D39ECF653B77D064
:107F20009DE9E40BD242C5A8A133321656A311F144
:107F30006F4543152DD3188314DF95809916649DE2
:107F40001164EEAB10FC1450BB4E89AF95774B100B
:107F50006B8EFAA59F109AE8F5D0FE275021E80510
:107F6000E88F3594019BA1E1E94661DF2DD09E1693
:107F70001A32EED18AFE5BCAC4C2180C9DB6F2C298
:107F8000803CCDAA889751B356A5BC444F555ACCD6
:107F9000CE70D778ED946639A2AB1C37E9A80219E8
:107FA000AC1D9E17FC78D808AD66AD03C419CEBFD2
:107FB00055FE27AA21B7D6D3973B4891D31343FD4B
:107FC00059D45D73AEDCCC488637BEDAA504B2F175
:107FD000DF8269FFE22CBEA3166AE9A6285D62BEB5
:107FE00007027C86DB8CA12E30BCB0D95E0B56E03C
:107FF0007E219CC4D7800C17819841DC8BBD0CEE90
:108000008D0D1733DDDC4B98310BF5F933BD0B418A
:1080100056EB0140D29CDEC54AF1C906AD8EE9E0BF
:10802000178E22C7A78B698C6C9989D8674D35B29A
:10803000852FEA4CAB870176CF3FE6CBBCAEB200D2
:108040007A3944E3B29C718FAF5660463D3CC762BB
:108050009AE2DD0821162908CF597A2CFA3A119FA5
:108060005A86CAFBDCC330C1E98C840355336A06E7
:1080700078A316653735F5EC89C14198939EC28E79
:10808000BEBDC7E0781C093A85B4088D4CB85DD8F0
:10809000E2C167D0BA9BB8587159DF95880BDAF8FE
:1080A00014C263E309769D6DE1153F746315BEEE5E
:1080B000C578080F7DEB52AA9EB057C7D3E72E01B3
:1080C000B10D3AE6749F83BE623A5F93EDD4D6A0B9
:1080D000302F119A99E1FF0BD269301B9880698D7E
:1080E0008FF891D439002B831C67C03D96AE9BED71
:1080F0007F9A8E6AB51C37B997B237759C2AC19D95
:108100000D276C77669686FECF22A0A57ABAAD229F
:10811000402D0F9CA60701A9B6A19A8B523EA0BD87
:10812000A5A249B1A58586BA2E8894DBD0A4A2DE8B
:10813000E98C2452969C553A7BD9BA206021E7F904
:10814000EB2103F90A21DD7BA71732A69C781C6777
:10815000318DCF6644AEAFDDCA6468F5D8DDD64454
:108160009EB00D2D0B6A559EA00BE6F3AB0E792247
:1081700007AB17B64663AEF997FAC5256C54051ED2
:10818000A159CF70007FD45F8184971B45C4CFEF86
:10819000A5ECDCFBBEBB4EB742A0056376333F2B9C
:1081A000639E98899740295D0FC38082340781932D
:1081B000A8E291E84C980DA7D9472187A901F60FAD
:1081C000871F5E228D3CA169F95A3FF88008234041
:1081D0005B0F28803A63D62BB20B665A05904EC7C8
:1081E000FC20817CD472112CDB74AB86F1C9A7AF63
:1081F000412293954E2F99E02E2D13F03526459070
:1082000014A5326C10A2346E2ABEBA4A15B3A1B2BC
:1082100073B8BF8F840A512B6DD365286818E64761
:10822000DEF8CA5171FA784F39FF9AAF91034C0CBE
:10823000DCE8B2F721A30D7F60FFF38E0885A7CAA3
:10824000AB918C15685A3BE6A649929B4B15CA65C3
:10825000CD3ED30949EA0DE377845F1B0350E9ED76
:10826000EE0D96BE9081AC8692A1FAB95F4B29EED5
:108270004D78010C467880C0E1092C0E5D017863D1
:1082800047B6BA5C1569FF5D21B20A0E22EFE7FB23
:10829000D05D48B3BFB5528B99331ECCB7728E3DBB
:1082A000068662F4943E2F719BD08C37CE50CCDD85
:1082B000D889FB51307D21CBE04DF5EBE90D79C735
:1082C0004E2C61A2DEE2C469A221E541746088A956
:1082D0001A4BA6282A8F40DA19B655DA948F0FC0A8
:1082E0006336FA7E087B2E0D55912EAA0775F4B5DC
:1082F000F3D24A68D636537213B0ED855E6BAA048A
:108300001193B64F6A8C50C95DC9D0F91B7E5DC20E
:10831000E1E8791900940293F14A1D912248321F35
:108320008D6847CB0A89097DC10B629DC09944B80D
:1083300001AA321612912CAFDBF865071F51382CB9
:10834000013BD646D53403FCEDC761A1F26EFD9F1B
:10835000814BD02B4934FF89E4F84BDC01488E6314
:1083600098AFEA2AB6D9F9CA7C2587026E5BB7A80E
:10837000FDCE627EF3094FE8811BD0BB7780E758C2
:1083800028BB8243C1DC94289D3F0F411E8758B112
:10839000B570A8E038219500A35880C749733B6D9C
:1083A000A12B74A2E547ADAB9A2928CD33B7D07382
:1083B000CDADBAC47D70A7F69B55302B20968CB6F8
:1083C000D4DADEC2F8DA959E09588FB3FC32241055
:1083D000E2DD9B2560602F62E4737B008387161BC0
:1083E000CFCEFF50E78AB03BC5E3FF7DB85E369F36
:1083F000E5CC5E8DA84C8AECF07D28BCBC5A1930C7
:1084000072ED3A4707F364C2335994048F199DF310
:10841000C9CAA96B9896F1FF32F5AD257391E8743E
:1084200029E33B8BC502881F28DFC333FAFE34A340
:108430003824A82BE5B8D43CF2A14EEC1069431ABD
:108440005B5136EC5878A14C4A9A2EBF7B2D98D7B9
:1084500070610C4BDF5BEADCEE48A2AEF49D8D64EC
:108460002ECBEFBB8C3B51752CD489B6E40B6D61E0
:108470002218FB85C0AE3A774A7A31C26EC94D25C3
:1084800029F0515A27F6392154E8B76563444BFC6B
:10849000F89F9FAD873D2BE745EB234BB4C05708B2
:1084A0008BC7897DFE33223C4D32CEBA4A4B5800F1
:1084B0009DF89111AC527820068A29F62CA1886487
:1084C000FCA837481EBCEA8A97640CC9A5A00A0418
:1084D0008B327E607CEC560E39B53AA3CEBF6E5619
:1084E000CAECE1EF6FA19C9B9A8EDB9D297825D881
:1084F000A4A65CAD1A34E35EE44349B05197FE0C88
:1085000093D916B98DE7D62FFBD8CDF35F58EB5F23
:10851000095C666740A6D15A04C3BC25145A6A1F79
:108520000E80321A7F8328E94AA4AAC0537C022D08
:10853000C0B984D929235FC548D1C2854700E39AD1
:10854000C3ECEF6673B19746A71A14282BB15800F5
:108550009EC835180ABC050DD708B30F3C239913E4
:108560003B3B9036BF5D2DF4CE18AAF9F72AC838E8
:10857000CCF96DE93C23CD84CF65BB3B2FEF8D2C2F
:108580006B97D6EC0DA5FE92CC80FBC7E8D5D397B0
:10859000529299F0768AB2CDC7FE0719124ECCC816
:1085A0003A952DEA5AFBAD98BE96BD22ED5E725605
:1085B0003ABA1BCC63E7393C1E0018E278D9BDE516
:1085C000AEFEFB7C8D1EE8FD5E520D5136293A450C
:1085D0004472924ADDB2C93BEFDC6913CD80363A72
:1085E000EA527745D16D330C41ADA1ED97D0EFFE46
:1085F000661181B80DF1E267F8671D8F61BCDA473B
:108600001598976B232F1AD6CA6DCF8C8EE3BAD0EC
:108610006EF8F16653E723BE0B26386514FB391557
:1086200001CB9595A399E6D24C03670CFDE2FA497C
:10863000EB6627310EDAD3F8198E42CCBEC9B1C72A
:108640006122B908570C1DDB238A7231B208245805
:108650000A13122384FB7817EF8D4D4977C4D33466
:10866000E4384F4A0D1A810F68BC500B15EF404A91
:1086700000944B8BEBCB0AD457090C307B5FFF7314
:1086800090ABDBA85F68D7FEECF66018FF11E190B5
:10869000D999B9CAB62040750E4AFE9F141F136FB0
:1086A000BA7DCA3A76C55B442DE77DF695C4BCA772
:1086B00050259F50B700C6DBE77193A28384C8851D
:1086C00002AB7D9B74067B51313A14E4C8CB582F22
:1086D0007F7C33FB0FC56651F810BA9391206B7104
:1086E000EBCDD2292D8760CAF8CDBD02B8716228C2
:1086F000A4C3E9A10A758AE6498D6ECF6987F62978
:108700003A4E39E6DB73AEA2F8977B4D73BA35105B
:10871000AB6B47074A421D60B1503EB6F5A5A1BFFD
:108720000A6D0DA718647769284BA3369F2932A7D5
:108730007B5E085A0F30BB9037140AAD3519DD1F28
:10874000688B5AAEFF48F8588B55B4BD736D42E73D
:108750009356A59DDA30BE80A08408FC23A95B4215
:108760004A68C78AB7B4D8BFD15D274FD06CB42C44
:108770004FBDE625DC69C41079F09A59B2843A38C5
:108780009460645ACC13BE18A986BCDBE3A53AC832
:10879000484A315FBF4BBE55A543D43661E0F77DF3
:1087A0009F7DDFA50B3BE51D200FF183BCAA35B0F3
:1087B0003591B3F10165DA394A65877C32704C48EE
:1087C000E79E8F4B40D3DAAC2DF5F3F1501E230713
:1087D0000A80579D80E3367754DACC45A8F7897F25
:1087E0000B8B62FDA172734B362DA95D417F984EB4
:1087F000BFBB7D1B71D1B5CAFA27BF6D03204052A4
:1088000023C2E3055FB43537222CA495E6CCF7C02C
:10881000B70D2D62F245091E05A3364DAE5B05B1BD
:10882000141537C40EA2B617CEE7BE1B4FF1647104
:10883000055C5706DF1AFAE9AE6513676C26988D5A
:10884000FD245096BCC705FBB6D213615508390B01
:10885000B6C9175E377A73EF3F9732D0321DEBC738
:108860008C70ED4E36193D0F38A40FA46FA2968A76
:108870007611A9D68ED89DFB80A50740AD213F4239
:10888000ADDA10AC6A08FD75EDFA8A12F305AE3563
:10889000764140CAF38D5C053A230E030BEADC6A8D
:1088A00057F2A80E9A44D2241778DB9A18C8D93305
:1088B000C169DA3DC97A1B969E9F120CC5A493B379
:1088C000397E54CA4A8F88DEF5476AA56C63003644
:1088D000F2262A15CAD86A7D00EC3EFD73FA9B1D6C
:1088E0005A28FC4B2F463AE34953DB9E4647155B1B
:1088F0000D93C43D8920478D7DEC329F1FEA6B208C
:10890000118CB91E29137E970FAD6BD5BF9970CF0F
:10891000B836CE3313FB094E0A35C87F21A92DD9AD
:1089200076F8621590AF81E0F0DD30414F160149D5
:10893000467EC7B92F48DF8BD78FA500DA937E2EEE
:1089400034DB1F71183E417E602420A8E54B267859
:10895000CD53AE2DF31E019A5916DFD8B2FD9EC03D
:10896000F91E986936D28C314EF10D78C890733863
:10897000FCE95CDC0DC511B987F17A4F6A3BFB8AD3
:1089800070D9E2B56F49A59A145FE02EA05A8F7393
:108990002E68046D8106C0A448E971314800973AF9
:1089A0009BDF5A6DF95F051556BD90452D2B3A9505
:1089B000E671E0A5CF68A173AC8E30C5CC6C533D99
:1089C0006E33D09C3D9B22336A2DEDA51770FBF7CB
:1089D000142A109ED6B7EE06125629D14CFB44F04D
:1089E000FECABDE13D9D30814CC838D7FD13361A13
:1089F0008EC6198537A91E5378413B28DE3DABE171
:108A0000374D960FC69C278AC37114DA14C1A0FD96
:108A10008278312EA0667ACA195C61C2BBCCE3C2EF
:108A2000D4575B4F7208744BA3019C2E172C0DF189
:108A30009D1E438665FBBD8F251F11A3383D42A4B3
:108A4000195E14403D28737A8D460A96D53A8A52AB
:108A5000453240DFB7AA179902CBC899813150C57A
:108A6000157E4B89BD025981630B3C5548058D8CA1
:108A7000698647908C6E40058FF728B488AE0C430A
:108A8000DCD31F4A2C0DB850FCBF57079620E137A6
:108A9000F416F1947E35A165B6F740FBF3B54418A2
:108AA0004D509E4B1004818DFF95A737FB40154F0D
:108AB000B6B926DD2196246AE3E2201D78AF87C788
:108AC000F82CA8E82BF8FD8BA15F05FCCEF03CA2AA
:108AD00012F3CFC5E7C124D1BB09B9EAB8B701A7E2
:108AE00086B5727E39B1008588FE478EFDCCFAB618
:108AF0009F0B7EA504381ECFCEF9357F8EF6096F09
:108B00007E323C27D4A88A501304D609555A7B0CD0
:108B10007B37CC6E021737B85A59C37E0004E8D6AB
:108B2000FB0D7F9C3CDFCB6B1B7818FE217A8F926C
:108B30002B7A227DE40D5B374D54B7EF58CFE22BF3
:108B400078520E6506C854370CC9D6F6BA90BBE504
:108B50005EA0A48BA6507B0F942F7941FFE18F0874
:108B6000DB96843460F7703F1EC7B28FBF9F0E0242
:108B700010A579B298B136A5EC1C2482C6E18E0905
:108B8000BB5D38C4DC6377AA9BF33A1AD223B41CCA
:108B9000458E577B95F6B11F901A0EBF05012D75B6
:108BA0006A3BB6D7E55E3B8976025B6E062820738A
:108BB000FDC6448637D52802A73994B1BF05EA9B84
:108BC0009C20AB8FFC169E5007A8EED4116F0CEDC5
:108BD0003861D839A7253F6B600AEDA86E87AAC80F
:108BE000F36C637738AE91F9DD1F3DFA3721257DAF
:108BF0009265B704371967A1E3A571B849ED6B75A4
:108C00004AF82A5A4F69375CEC5C64F13F1DAB9817
:108C100002DE197C97DB53B90E4B9BF2EF3EA6AFF9
:108C200063F9487FA11E8B7E7F2DD994E93D6E8527
:108C30005B099485E634F79F56DC6AA8BBB70F132F
:108C400037D2DC4F2E272B91F1C878E4588CC2D054
:108C5000579F10AA22998F6EE52DC8B90B2093EE6D
:108C6000EAD53F6CAF5A4EC868FA93D95CCFEBDFB8
:108C70006E8401B0463216293B5AC923DF40CEEE3E
:108C800065AA2D316AE91811F10106A59F31CD9D24
:108C90002CA2F2FA706E2DC6D097F3897C2E0FEEBF
:108CA000049B81AE8FDBB3DCD21AE270FD4A71C93E
:108CB000C6DD09ACD89A999422320105BB966DB9EC
:108CC0004FAEE9395BD83E113774F5C87329665E3B
:108CD00052F3059361F97B4170CCF07B88BDC6BA35
:108CE00045AEE260AE2E30D5476BFFEA1CA842EEDF
:108CF00020609CFFEEE2D7B04A1C7C8E691F64C9DD
:108D0000E59D596FF5B16F600E92AF195DA36D854A
:108D1000835A65322578243049933BCAE395B3D909
:108D2000999167217B099D86ABABF561F5E786E4F8
:108D30005CF033FC3BAE932202125D40BEE6BC5EAB
:108D40007BBD1FEF4B80ED71965094853B19A404B9
:108D500058B9ABB78B88C908A689AF8B2FBCE98AF5
:108D60009FFF5E9DA9F5055751E887AF1307CE51C8
:108D7000B61609C2F6D88EEEB16E44A784BBDB5797
:108D80001DF3587726B24C5E194BAAB171588E9FCD
:108D9000AC153B78C40A1BD7E15DB8A179BFD99D5A
:108DA000E74E392237D9DB556A90834E2D88C6CBE2
:108DB000B6D73A5FFBB9B0A42362D33A80A8CF619B
:108DC000B5C2336254BD6B015AD9A0C13F4CB2EA5F
:108DD00053AE8C1D33A72F70135DA52232DFFCF438
:108DE000F56CEA794C76A1EC25030F2451E378B1B8
:108DF00099E1801F003BD70E0D59DE296CF39D10C1
:108E00005950C3B8873B631A52FF6BB93778D39078
:108E10003330B8EFEDF2A917E49350CA1835CA0DF4
:108E20009515BFA15F6F8DDE889A7882D3DF4A8463
:108E3000FE2F166F95EBF7C2A6221465F77726A0D2
:108E4000F27817FD5FAE6183D2A133BF5FD85AFBC2
:108E50001D9F5454DBA6D7882F2D6FFE37D3DD40DE
:108E6000FAE066EAFC6C89888AE6CFE33EAB9E11A5
:108E7000DC1DC57F24F7031DAC7C22D7A07653CA26
:108E8000EB8DC13F32E25A3F16AAE378322652896F
:108E9000A55F0BC1B6968D4DC244CA24FB74D8039E
:108EA0001C7B8653D1C9E60F5778EF060EDEBA2732
:108EB000A9AED2C2252B75DD1F8AD4A2B361CA66C2
:108EC0004C24DEBEB50A0503F85E3F67232CC83D7F
:108ED000E4D06AC314BC37791AA1059E84CA1D0C5C
:108EE000E8EACF3AB41C644715ADB38440EAB067F2
:108EF0003BDBDFEAE6B2AEADD44CC31DF2BAF6728C
:108F0000061D1CDFA84A8A3593FCAD9496BDB8BEF9
:108F100093F504EA5002927142445D5DCAEF97CD29
:108F2000DFF4B440321B146C42A15C69673E12E668
:108F30009FF1B1AA04676716AD1AD4EE9753CB041C
:108F4000E78325B1B4AA42595CCDA1E258C35C368F
:108F500048BF8ADDEF320F743A491D1993D524F6C4
:108F60004FED0D3D26C42F86416BE5D2DD58EFB69F
:108F7000B9290741ABE0D27D3381FA8783C89CA031
:108F800092950EB31E45C3FACDBCC0A3EA02992741
:108F900009CFF653D3966C3C40FFF16AD79C9BE90E
:108FA0009CCD1F06B467F9B51BA7953CC142C566A9
:108FB00005307086D2E7D2C238F0775A617116B8A0
:108FC00001857CCC15BACD51D4BBFE231AE29B425D
:108FD000D2DA86BEA4C430BA217A27A71D6DE9EE85
:108FE0003BA8DAF0DFFD35BDD9CA87320CF8C8A836
:108FF000EA3193FD0B729CB678DEF5B85ABFA963CF
:10900000C4BB8BD9DD08AE9FF5683D1AE55BB3069E
:10901000387AF1935DAE2BFE7B6C8E2DD1A9407F0B
:109020007CF269974CFF1F7141D94D7346FA6A086B
:10903000329ADDFE0313DD4D1938B95F72E30F0973
:109040000B533A8A8DDB970A58C68EE538999E07EE
:1090500038B19DB3E3C8F6802A1FA9A6ABB14E8FE5
:10906000A6DEC3E1683F322A5C915D69EE5531733B
:109070007F8B4E2A781BD2C66EFE75BF327CE5C54B
:10908000F41E6767ADF2558304F4C78962533A1F33
:1090900018BF1B09E5C14400CBB3BA0E63CB7925D9
:1090A000DAF12ED9E701B5DF367BB6BF9A5487A631
:1090B000FD094D1C192754EE34DE5D80D10EDC48CD
:1090C000661B34BE9C0E6CFCF6C29DE8BAE1816161
:1090D000C57CDE3225C3C85FE5041A0AAED4A5F10B
:1090E00015A078967C7A5230E004847F9CF5D939BB
:1090F0006F96C9C3BB10CEAB9DA98E48CD63CB265E
:10910000B133495E31A5E170496C84590A1443C8F2
:10911000B1C5C2D46AAFCE3C275FCEDABCE9AC1190
:109120007C2E937B25FF658BAFA7D3B12AE42B0060
:10913000301A58D52ED6BB8CB2B3F8C6E219936B51
:10914000A6809CC7A135D0695FB4B8C1EA58BBF20C
:109150002FF6E88D6913FEA559735C8D49EA77B344
:10916000DBB77DEE610642BCDCF0DCBFA3C4ECA83B
:10917000A5D09DD76568A15E0D63D4D1DF3F474C74
:10918000E512CBF72FCDF7B9D7255BE41990C0CD09
:1091900082EB40A12B3FE132A6F45C4B81DC1863EB
:1091A000D110301D1FA7A1547D788E0C546D2DB0A9
:1091B000B4243AC18A3432C7F71A590CB7394AFF76
:1091C0000BD6E8239CFA6DDFBA8C30A71FAF1C09C1
:1091D000FA26E040044D9D2A731DC8DD14EF0BB242
:1091E000EEF1C2D4EED8B645DDE3BC6CD167B0B2C7
:1091F000D6E8F00F9070F2954C729E637616A0B68A
:1092000056E1F944DAAC845BAF266CDA57F00C5DBA
:1092100085AB08CF758AA47A6EDC409957FD089714
:109220001386B23B18256833AF197595B76991F469
:10923000C74AA36E3D581CE2EAA197A43D4C0075B5
:109240003999AA7362DA2928B53274C10E3D4358A0
:109250009B1C19FD868974CE92FDD9A00EEA5A6A2C
:1092600098AA0FFCB10B6D0A78F414D2C445C41649
:109270009A9ED79E6300326839BCCEE6265DB79FC2
:109280002717CEDD3CED70BF2FA7DC4FF0BDEBA460
:109290008A42E41A0CEE529477119BA7E10D07A9BC
:1092A000EE33D33C4EF3C5DA72D61D5FA16EBD8698
:1092B000CAB318E4EC9FD13C8915212E5E031882B5
:1092C000ED2D7351A8DB14FED71A867B187E2A6712
:1092D000D54B1065DADAE80190715A729AB513E647
:1092E000B169BEE60981902C44B2AE47F5C94D3153
:1092F000B2288C882C2FA71C740879D99EC84328C3
:109300001CB8A9DBCEA139EC37EB4A52837732FF88
:10931000001CAF0304050A08060BFF0209070D0134
:109320000C00FF2025692025692025692D2569006D
:10933000202025633A256900202020205F5F7C00E3
:109340002C00610044697370206F66660D0A005539
:109350005345520046004700424547494E0052419E
:109360004400442E4D59005052474D00555345522C
:109370002020200066202000672020004245474929
:109380004E20202020200052414420202000442E46
:109390004D592020200043202020000D0C205AD5BC
:1093A0004D00000D0C205AD05100000500000003B4
:1093B0000720610F4D0000FFFFFFFF4D000000F18F
:1093C0004B000000000000BD18000064550000695B
:1093D00055000067550000FF000000B10D0000734C
:1093E0005500007D550000F556000000000000E12A
:1093F0000B00008F550000695500008556000000E5
:10940000000000810C00009B55000069550000A77A
:1094100055000001000000350E0000AA550000BAFA
:10942000550000A855000000000000090B0000C412
:1094300055000069550000CD55000002000000698C
:109440000B0000D0550000D9550000ED550000017B
:10945000000000A90B0000F0550000FC550000EED4
:1094600055000000000000090E00001056000069C1
:109470005500003156000000000000F50A000033DE
:1094800056000069550000F7560000FB560000FF2B
:1094900056000003570000075700000B5700000F4D
:1094A00057000054550000FFFFFFFF0F000000F4BD
:1094B000010000040103010201010411040F04175B
:1094C000041601180100006C9300007493000078EA
:1094D0009300007C93000056930000879300008E59
:1094E0009300009693000067930000081C242C440E
:1094F00048586C740502050804080B0804040501AB
:109500000504090809040608070206020402060108
:1095100006040701030803040C080D020C020302F1
:109520000C010C040D010D080D04080208080708C1
:109530000202070408010804090209010A080B02D3
:109540000A0201080A010A040B01020802041008B9
:10955000110210021108100110041101120212016F
:109560001302130812080F08120413011304140243
:109570001401150215081408170814041501150420
:109580001702170119081A02190216021901190403
:109590001A01160816041B021B081A0818021A04DE
:1095A0001B011B04180818040B0420202020202075
:1095B00020202020000000010000004F93000054F4
:1095C0009300005693000058930000569300005EED
:0F95D00093000062930000D356000067930000E1
:00000001FF
